:020000040800F2
:10000000981100200101000847380008FD28000869
:10001000453800084D0F0008AD62000800000000E0
:10002000000000000000000000000000FD48000883
:100030009F1A000800000000B53D0008094C0008A8
:100040001B010008A93B00081B0100081B01000858
:100050001B0100081B0100081B0100081B01000810
:100060001B0100081B0100081B0100081B01000800
:100070001B0100081B010008211500081B010008D6
:100080001B0100081B0100083D0700081B010008B8
:100090001B0100081B0100081B0100081B010008D0
:1000A000794C0008654D00081B0100081B01000881
:1000B000694D000851500008AD5200081B010008AE
:1000C0001B0100081B0100081B0100081B010008A0
:1000D0001B010008A55D00081B0100081B010008AA
:1000E0001B0100081B0100081B010008DFF80CD0F1
:1000F00000F0E6FA004800476974000898110020F3
:100100000648804706480047FEE7FEE7FEE7FEE7B1
:10011000FEE7FEE7FEE7FEE7FEE7FEE7294C000804
:10012000ED0000082DE9F0410024061B254671F181
:10013000000605DA01240027D0EB070067EB010178
:10014000161E73F1000605DA0027D2EB070201251F
:1001500067EB030300F0D0F986460E4617469C462F
:10016000AC4204D00025D0EB050E65EB010624B1AE
:100170000020D2EB000760EB030C704631463A4694
:100180006346BDE8F08140EA01039B0703D009E024
:1001900008C9121F08C0042AFAD203E011F8013B73
:1001A00000F8013B521EF9D2704780EA010210B5F7
:1001B00002F00043400022D04A001FD0010E01EBA4
:1001C0001261C0F35600C2F3560240F4000042F43C
:1001D0000002A0FB022000047F39140400D0401C60
:1001E00050EA124001D44000491EC2B20C0604EB92
:1001F000D010401C4008802A02D003E0002010BD2F
:1002000020F00100002900DA0020184310BD2DE97C
:10021000FE4F81EA030404F0004421F00041009401
:100220004FF0000B23F0004350EA01045ED052EA85
:1002300003045BD0C3F30A54C1F30A552C44A4F25F
:10024000F3340194A0FB0254C1F3130141F4801173
:10025000C3F3130343F4801301FB024400FB034E7A
:10026000840A970A44EA815447EA8357A4FB076843
:1002700002958D0A05FB07854FEA932C04FB0C546D
:100280002705029D4FEA065847EA1637B5EB0805E1
:100290006EEB070C870E920E47EA811742EA831233
:1002A000A7FB0201B6EB0B0164EB00042B0D43EA44
:1002B0000C335E1844EB1C50DA465146E7FB020152
:1002C000C5F313044FEA0B3343EA14534FEA0432E5
:1002D000019C43EA0603A4F10C040294009CCDE9BE
:1002E00000B400F09FF903B0BDE8F08F0020014694
:1002F000F9E72DE9F04D81EA030404F0004B21F009
:10030000004514464FF0000A23F0004150EA050270
:1003100020D054EA01021DD0C5F30A570246C5F3A6
:100320001303C1F31300C1F30A5640F4801543F4DC
:100330008013A7EB0608101BD64608F2FD3873EBB6
:10034000050002D308F1010801E092185B41B8F101
:10035000000F03DA00200146BDE8F08D00204FF4C5
:100360008011064684460EE0171B73EB050705D384
:10037000121B63EB050306434CEA010C49084FEAE4
:10038000300092185B4150EA0107EDD152EA0300B8
:1003900012D082EA040083EA0501084305D0101B4D
:1003A000AB4106D20122002306E000224FF00043B9
:1003B00002E06FF0010253101AEB06004CEB0851FB
:1003C00010EB0A0041EB0B01BDE8F04D00F01BB94A
:1003D00070B521F0004303430CD0C1F30A5500244B
:1003E000D5EB040564EB0403D617AD1AB34102DB69
:1003F0000020014670BD201841EB025170BDC10FB5
:1004000080EAE0700844CA079623002100F0CDB8C6
:1004100096230022114600F0C8B80EB5C10F80EA3D
:10042000E0700844CA07002140F233438DE80E0013
:100430000A460B4600F0F6F803B000BD0EB540F2D8
:10044000334102910021CDE900110A460B4600F02C
:10045000E9F803B000BD00F0004220F00040C10DFB
:10046000C0F3160040F400007F2901DA0020704735
:10047000962903DCC1F19601C84001E09639884015
:10048000002AF4D04042704770B5C1F30A5201F01F
:1004900000450024C1F3130140F2FF3341F4801101
:1004A0009A4201DA002070BD40F233439A42A2F230
:1004B000334203DC524200F05FF800E090402C43EE
:1004C000F1D0404270BDC1F30A5210B5C1F313011F
:1004D00040F2FF3341F480119A4201DA002010BD4E
:1004E00040F233439A42A2F2334203DC524200F01C
:1004F00043F810BD904010BD2DE9F05F0546002087
:1005000092469B4688460646814640241BE0284684
:1005100041464746224600F02FF853465A46C01A35
:10052000914110D311461846224600F016F82D1AB4
:1005300067EB01084F4622460120002100F00DF82C
:1005400017EB00094E41201EA4F10104DFDC4846F0
:1005500031462A464346BDE8F09F202A04DB203A74
:1005600000FA02F1002070479140C2F1200320FA06
:1005700003F3194390407047202A04DB203A21FA04
:1005800002F00021704721FA02F3D040C2F12002AC
:1005900091400843194670470029A8BF7047401C86
:1005A000490008BF20F00100704710B4B0FA80FC89
:1005B00000FA0CF050EA010404BF10BC704749B1C6
:1005C000CCF1200421FA04F411FA0CF118BF012136
:1005D00021430843A3EB0C01CB1D4FEA00614FEA16
:1005E000102042BF002010BC704700EBC3501044E5
:1005F0000029A4BF10BC7047401C490008BF20F070
:10060000010010BC704710B5141E73F1000408DA25
:10061000401C41F1000192185B411A4301D120F0C6
:10062000010010BD2DE9F04D92469B4611B1B1FA83
:1006300081F202E0B0FA80F220329046FFF78DFF9F
:1006400004460F4640EA0A0041EA0B0153465A4667
:10065000084313D0114653EA010019D0C8F14002F3
:100660005046FFF789FF05460E465046594642461A
:10067000FFF773FF084305D0012004E02046394608
:10068000BDE8F08D0020054346EAE0762C43374371
:100690000A986305E40AA0EB08000022FD0A44EA78
:1006A00047540A3002D500200146E9E70105101938
:1006B0006941DDE9084500196941BDE8F04DA2E74F
:1006C000064C074D06E0E06840F0010394E807009F
:1006D00098471034AC42F6D3FFF70CFD3C9300086A
:1006E0005C93000870B58C1810F8015B15F00703D7
:1006F00001D110F8013B2A1106D110F8012B03E0BB
:1007000010F8016B01F8016B5B1EF9D12B0705D4C2
:100710000023521E0DD401F8013BFAE710F8013B0B
:10072000CB1A921C03E013F8015B01F8015B521E27
:10073000F9D5A142D8D3002070BD000070B54C4C53
:100740004FF490652946204600F015FA002863D042
:100750002946204600F0A2F846490888401C088037
:100760000121204600F0E6FA434942F21072B1F846
:100770005800904202D2401CA1F8580007F05CF8E3
:100780003E4DB5F91410B5F9120005F02FFF3C4CA1
:10079000A5F856002080A16820468847A088A5F8C3
:1007A000580003F0B9F807F043F9364E364C30786C
:1007B000082832D045F6AC30606042F6EF60A060A9
:1007C00042F2C400E0603148008A2080208E6080C0
:1007D000A16B2D488847208E40F21C7180002C4C64
:1007E00000EB81006887207A4FF0000540071DD597
:1007F00001F0E4FA274949F6A2400880264840F271
:100800001A62C188491C89B2C180914204D3A1688F
:1008100021F00401A160C58070BD41F21300606049
:100820004FF48060A06040F61B50CBE730780A2878
:1008300018D2DFE800F0170613050A050D1711138B
:10084000EAE7BDE8704006F07BB808F05FF805E025
:10085000BDE8704002F0AABD06F0F8FBBDE87040AC
:1008600007F03EBA00F00AFC84F8B65070BD0000F4
:1008700000240140200700204C01002064000020DB
:100880004007002017070020E40000200402002099
:10089000B4020020442C0140880900206FEA112195
:1008A000016070470029816802D041F0010101E038
:1008B00021F00101816070470029816802D041F474
:1008C000807101E021F48071816070472DE9F04171
:1008D000824E92B0304600F00BF90BA800F039FAC6
:1008E00001214FF4C06003F0F9FA00248DF8314083
:1008F0004FF46020CDE90D044FF4A0204FF009081B
:100900000B9001278DF83C808DF830700BA9304694
:1009100000F080F9724D8DF831408DF830708DF80F
:100920003C700BA9284600F075F9052301220F2120
:10093000304600F0C0F9022205231146304600F08F
:10094000BAF9052303220021304600F0B4F905234B
:1009500004220121304600F0AEF905231A460B218E
:10096000304600F0A8F9052306220421304600F0A5
:10097000A2F9052307220821304600F09CF905233F
:1009800008220321304600F096F9052309220A21A6
:10099000304600F090F90121304600F084F9012141
:1009A000284600F080F901231A460521304600F060
:1009B00055F901231A460621284600F04FF9002177
:1009C000304600F0CBF84FF4E041284600F0C6F87E
:1009D0000121304600F0B8F80121284600F0B4F8B3
:1009E0000121304600F0A6F80121284600F0A2F8C7
:1009F0000121304600F09EF90121284600F09AF9C5
:100A000040F61451374804F028FF12208DF84000BA
:100A100002208DF841008DF842408DF8437010A8F7
:100A200002F03EFF01224FF49061304600F0E8F8FA
:100A300001213046FFF740FF01213046FFF732FF2A
:100A400001212846FFF72EFF304600F06EF93046B0
:100A500000F09FF80028FAD1304600F075F93046D2
:100A600000F082F80028FAD1284600F05EF9284606
:100A700000F08FF80028FAD1284600F065F92846E2
:100A800000F072F80028FAD10121084603F002FABA
:100A9000154D284600F080FD684600F028FE0F48FE
:100AA00001A94C300090114881E811018020CDE966
:100AB00004404000069080000790202008904FF4EA
:100AC0004050CDE909046946284600F0F3FD0121B4
:100AD000284600F055FD12B0BDE8F0810024014029
:100AE00000280140002C014008000240C402002000
:100AF0000D4910B5884202D1012144150AE00B4985
:100B0000884202D10121041504E0094988420AD132
:100B10000121CC03204603F0EDF92046BDE810404A
:100B2000002103F0E7B910BD002401400028014076
:100B3000003C01400029816802D041F4801101E0AD
:100B400021F48011816070470029816802D041F44E
:100B5000004101E021F4004181607047826822F485
:100B6000E0420A43826070470146002089684907D5
:100B700000D50120704710B50246002054680B0ACA
:100B8000C9B20C401168194202D0002C00D00120DB
:100B900010BD014600208968090700D50120704773
:100BA00038B501211C2003F099F9FF20ADF80000B1
:100BB00000248DF8034003258DF8025069460D4846
:100BC00001F00CFB0120ADF800008DF803408DF81A
:100BD00002506946084801F001FB2320ADF80000EF
:100BE0008DF803408DF802506946044801F0F6FA8A
:100BF00038BD000000080140000C01400010014019
:100C0000002A4268C9B201D00A4300E08A43426028
:100C10007047000010B542680E4B0C791A400B6803
:100C200042EA04221343436083680B4A1340D1E92C
:100C3000024222434C7943EA44031A438260C26A67
:100C4000097C22F47002491EC9B242EA0151C16214
:100C500010BD0000FFFEF0FFFDF7F1FF70B50724A7
:100C600009290AD9C568A1F10A0606EB4606B4406F
:100C7000A543B3401D43C56007E0056901EB41068C
:100C8000B440A543B3401D430561836BC3F30154D6
:100C9000121B921C02EB82041F22A2409343A1402C
:100CA0000B43836370BD826B491E22F4401242EAFB
:100CB00001518163704770B5072409290AD9C568B5
:100CC000A1F10A0606EB4606B440A543B3401D4316
:100CD000C56007E0056901EB4106B440A543B34098
:100CE0001D4305611F23072A09D2446B521E02EBE4
:100CF000820293409C4391400C43446370BD0D2A93
:100D000009D2046BD21F02EB820293409C439140B4
:100D10000C43046370BDC46A0D3A02EB8202934037
:100D20009C4391400C43C46270BD816841F008014E
:100D3000816070470029816802D041F4A00101E080
:100D400021F4A00181607047816841F00401816055
:100D5000704700210160017141718160C160012112
:100D60000174704770B51E4C214694F83800B1F8F4
:100D7000425006281ED9B4F84A10B4F84C00A1EB32
:100D8000000202F10902122A04D8FFF757FB0022E1
:100D9000144B0AE0884204D2FFF750FB0022124BAA
:100DA00003E0FFF74BFB0022104BFFF730FAFFF791
:100DB0008AFB09E005D12846FFF740FB0C4A0D4BA2
:100DC000F3E70D4951F82000C5EB45116063B0EB26
:100DD000410F03D9C5EB45104000606370BD0000B2
:100DE000640400200000344000003340000035401F
:100DF0006766666666E64B40E48A000810B50C4CF0
:100E00002078400713D5FFF7ADFF0A49A08E088070
:100E100008483038018821F010010180001F018846
:100E200041F010010180207820F00400207010BDF6
:100E30006404002040040040F0B4184816494FF400
:100E40009677436C08468A68046815485FEAC25C76
:100E500042F00806007822F008054FEA047415D520
:100E6000002C08DB120714D408B1082811D1BB42AA
:100E70000FDA8E6007E012070BD508B1082808D1F9
:100E8000BB4206DA8D60F0BC05F0E2BE002CF2DA5F
:100E9000E8E7F0BC70470000B40200204C010020DD
:100EA00017070020012180F82E104FF4AF61018652
:100EB0001F21418645F271518186704770B5064603
:100EC0004089204B204C4FF48071002580B362880C
:100ED0007AB1012A0CD1E188491C89B2E1803289BA
:100EE000914205D36580E580FF2801D0401E7081C6
:100EF00070BD70882288904201D9012200E0002252
:100F0000184601F0F4F97088B18801442088401C2B
:100F100080B220808142EBD82580A088401C80B21E
:100F2000A080F1888842E3D301206080A58070BD55
:100F3000FFE70022184601F0DAF9A580E580258058
:100F40006580F4E7000C0140D4050020FEE70000B6
:100F5000FCB505464FF6FF7600200C46ADF8006064
:100F600048F205078DF8040020E000BF15F8010BDA
:100F70008DF8040001A9084602F0F5F8BDF800005C
:100F80009DF8041080EA0120ADF800005FF0000039
:100F9000BDF800100A0402D587EA410101E006EA23
:100FA0004101401CADF800100828F1DB641EDDD2C1
:100FB0006946084602F0C1F8BDF80000FCBD00001B
:100FC0000246002004E000BF12F8013B1844C0B202
:100FD000491EF9D27047000070B5144A85B01088D8
:100FE0000024134901940094039420460494138828
:100FF00007E00D8B009E35440095CD8B019E354456
:10100000019515889D42F4D0401CC0B28028EED3D3
:101010000098411107484180848001984111064899
:1010200081830183818205B070BD0000200700200C
:10103000B4020020EE050020DC04002030B50E498B
:1010400002880A800C4A4388083A13800B1F808864
:1010500018802024151F2C800020401C80B273288B
:10106000FBD341F21110088044F64800108047F28B
:10107000480018802C8030BD202C0140114944F6D6
:1010800048000880091D46F648000880091D41F205
:10109000111008800B48001F018841F020010180D9
:1010A00009480021A0F86410A0F86210A0F86010B0
:1010B000A0F85E10A0F85C10A0F85A100348418117
:1010C00081827047182C0140B40200206400002087
:1010D0002DE9F047494B4A480021DA7A0778802AFF
:1010E00027F0010676D31C68464B02F01F0253F826
:1010F0002220454B14421A6802D042F0200201E03F
:1011000022F02002DFF804A11A60424CDFF8F8C098
:101110009AF80050DFF8F890B4F904409CF846C003
:10112000022D58D11D89C5F3C008C5F30025A84577
:1011300051D0354D303D95F80280B8F1000F06D002
:10114000B8F1010F0DD0B8F1020F49D120E011051F
:1011500046D5910644D40121A97027F004010170FD
:101160003EE016053CD496063AD57E0738D446882C
:101170007EBB4480002C09DD47F00501017002218F
:10118000A9702549B1F84410018229E0A97027E02F
:10119000C7880FB9002C12DC077B67450FD11F4FA2
:1011A000BF895FEA47780AD45FEA877807D45FEAA5
:1011B000427804D55FEA826801D5FF0710D0067037
:1011C0004180A9F8001041810182A970D9738AF881
:1011D000001005E00DE006704180A9F80010418183
:1011E000C48080F80CC0500960F3CB221A60BDE8BF
:1011F000F087067041804181F9E70000F405002086
:1012000070090020448F0008B40200201707002056
:1012100024010020EE0500204C010020C00A00201F
:101220002DE9F04796B000240C940D940E940F9481
:1012300072B69048816941F400718161816941F41D
:10124000806181614FF4004002F01AFE8A4D002156
:101250002846FFF731FB00212846FFF723FB874E86
:1012600000213046FFF71EFB854F0021384600F075
:1012700087F901204FF47041401C8842FCD3284676
:10128000FFF736FCB1463046FFF732FC384600F037
:1012900083F94FF46020CDE912048DF84540012018
:1012A0004FF004088DF8440010948DF8508010A978
:1012B0002846FFF7AFFC01231A4605212846FFF711
:1012C000FAFC0123022206212846FFF7F4FC012341
:1012D000032207212846FFF7EEFC012304220F21F9
:1012E0002846FFF7E8FC384600F056F9684600F05B
:1012F000FEF96148634E4C300090CDF80C80CDE98A
:1013000001648020CDE904404000069080000790F1
:10131000202008904FF44050CDE909046946384632
:1013200000F0C8F901212846FFF7C6FA0121384626
:1013300000F026F901212846FFF7B4FA47F23051B0
:1013400015941598401C15908842FAD3012128461F
:10135000FFF7F0FCADF82C40A04640F2DC5A4FF409
:10136000007420E05046CDF854801599491C159121
:101370008142FAD330880D9908440D9070880E99F7
:1013800008440E90B0880F9908440F90F0880C998B
:1013900008440C9001212846FFF7CCFCBDF82C0036
:1013A000401CADF82C00BDF82C00A042DAD30D98FB
:1013B000354A40F3CF1633480A3006830E9941F37D
:1013C000CF1444830F9941F3CF1383830C9941F3D6
:1013D000CF1CA0F804C0ACF5C05C40F2C371ACF502
:1013E0009B7C8C450ED2A6F5C856363E8E4209D25D
:1013F000A4F5C854363C8C4204D2A3F5C853363BFE
:101400008B4203D3D18841F48041D180D1884904F3
:1014100007D41E49028B21F85C2F428B4A80808BB7
:10142000888000212846FFF747FA0021384600F05F
:10143000A7F800212846FFF735FA00214C46484618
:10144000FFF730FA0220C102401C8842FCD3284634
:10145000FFF74EFB2046FFF74BFB384600F09CF8A9
:10146000FFF734FA0A493C20087062B616B0BDE8AE
:10147000F0870000001002400024014000280140D5
:10148000080002403A050020C00A0020200D00207C
:101490001407002070B5204B40F6C81441F2B70580
:1014A0005B6C48F6E6065C4305EBA4341B4D7343C6
:1014B0004EF6F61606EBA333C5E90443D460401A92
:1014C000536110609168884202DA4942884200DC28
:1014D000116010684343107E0341906A19189162AD
:1014E000506A814200DD9062916A106A814201DB9C
:1014F000084600E09062A86111684C43117C0C41E1
:1015000008412118B2F91C00884204DBB2F91A0024
:10151000884200DC08B270BD4C0100202801002088
:1015200010B54FF40054204600F0ACF8002813D05A
:101530000A49087840F008000870204600F014F8C6
:101540000021074800F01CF80648C17E012903D19C
:101550000021C1760121017710BD00008E06002018
:1015600044000240C40B0020C10002D502490860BB
:10157000704702494860704704040240000002407E
:101580000029016802D041F0010102E04FF6FE722D
:10159000114001607047000001684FF6FE72114073
:1015A00001600021016041608160C1603149314AC0
:1015B0000839904203D1486840F00F0006E02D4AF8
:1015C0001432904204D1486840F0F00048607047FF
:1015D000284A2832904203D1486840F47060F5E709
:1015E000244A3C32904203D1486840F47040EDE711
:1015F000204A5032904203D1486840F47020E5E719
:101600001C4A6432904203D1486840F47000DDE720
:10161000184A7832904203D1486840F07060D5E7AC
:10162000154A111F904203D1086840F00F0006E0F0
:10163000114A1432904204D1086840F0F00008606A
:1016400070470D4A2832904203D1086840F4706018
:10165000F5E7094A3C32904203D1086840F47040F3
:10166000EDE7054A50329042EAD1086840F4702014
:10167000E5E700000800024008040240406880B22C
:101680007047000001460020CA0001D5034A00E06F
:10169000034A12680A4200D0012070470004024049
:1016A00000000240002A026801D00A4300E08A4399
:1016B0000260704730B5036847F6F07293430C6AD6
:1016C0008A682243D1E904452C4322438C69224392
:1016D000CC6922434C6A22438C6A22431A4302603B
:1016E000CA6842600A6882604968C16030BD0021F2
:1016F000016041608160C160016141618161C161DE
:10170000016241628162704710B5114C8CB00021BA
:101710002046FFF735FF2046FFF73EFF0D480090BB
:101720000D480021CDE901016420CDE903018020AD
:10173000CDE905010791089109910A916946204672
:10174000FFF7B8FF01212046FFF71AFF0CB010BDCC
:101750005800024004380140B007002010B50121B4
:101760008CB0084602F096FB1E4C00212046FFF785
:1017700007FF2046FFF710FF1B4800901B48019011
:1017800000211020CDE902018020CDE9041006914E
:101790000791089109910A9169462046FFF78AFF4F
:1017A000012202212046FFF77DFF01218DF82F1035
:1017B00004208DF82D008DF82E100E208DF82C00B1
:1017C0000BA802F06DF80F208DF82C000BA802F08A
:1017D00067F801212046FFF7D3FEFFF795FF0CB015
:1017E00010BD000044000240043801404C070020B6
:1017F000F0B540F6AA222A49C284838B0C88E31AEA
:101800009BB20F2B0DD309888183037E00213BB14E
:10181000244BB3F90A40244B032C03DA818429E0DA
:101820008184F0BD214C2478022C02D0002CF5D00C
:10183000F0BD1F4C40F68B27656C1B4CA5F22D1696
:10184000BE42B4F9004017D2418B491C89B2418392
:101850006429EDD364214183B0F92410914201DA67
:1018600001EB22128284641C20B24FF400711880B4
:101870008842DDDB1980F0BD41F29416B542FADBF7
:10188000B0F92450002D02DDA5EB221200E0002269
:1018900082844183641E20B218800028EADDF0BDF6
:1018A00020070020640000206004002017070020AB
:1018B0004C01002010B50446B0F9020043F699111E
:1018C00048438113E06840F26662504301EBA03068
:1018D000E060B4F9001043F6991251438A1321696C
:1018E00040F26663594302EBA131216104F01EFE10
:1018F0006061A18840F6AB2208444010A0F5154174
:101900005539E062914205D9A0F5F851FF39521CD2
:1019100091421DD249F25451884202DDA0F5204087
:1019200002E0A0F5F850FF38206300EB400040F3E0
:101930004F002085B4F924104A42904201DA104643
:1019400002E0884200DD0846E083228461848AE068
:10195000A0F5FE42FF3A41F255518A4214D8A2F650
:10196000AA20206300EB400040F34F002085B4F92B
:1019700024205142E183884201DA084602E0904285
:1019800000DD1046404250E0A0F5D442AA3A8A4217
:1019900015D2A2F6AA20206300EB400040F34F01CD
:1019A0002185B4F924004242E2832084914201DA85
:1019B000104602E0814200DC0846608453E0A0F556
:1019C000AA42543A41F256539A4215D2A2F6AB209B
:1019D000206300EB400040F34F002085B4F9241051
:1019E0004A42904201DA104602E0884200DD084691
:1019F0004042E083218419E0A0F5804241F2545333
:101A00009A4215D2A2F6AA20206300EB400040F3D0
:101A10004F002085B4F92410E1834A42904201DA54
:101A2000104602E0884200DD0846208462841AE005
:101A3000A0F52852AB3A8A4215D2A2F6AA2020631A
:101A400000EB400040F34F012185B4F92400E0830E
:101A500042422284914201DA104602E0814200DCD7
:101A600008464042A9E7B4F91E0041420948B0F9CE
:101A7000000041438913E180B4F9201049424143F9
:101A800089132181B4F922104942414388136081AE
:101A900010BD0000600400200121017670477047EE
:101AA0001548164A4FF480410078042821D002F1ED
:101AB0003C03D08A9B88C01A00B22F2801DD001198
:101AC00008E0002801DD002007E00D4B984201DA14
:101AD000184602E0402800DD40209389184400B2F7
:101AE000884203DC40F26661884200DA0846908151
:101AF000704791817047000017070020DC04002028
:101B0000C0FEFFFF38B54B484B4902880B889A1A34
:101B100092B20F2A71D30988484C01804FF0FF011F
:101B2000E2884FF47A7355044FF4967002D516226A
:101B3000009103E0950403D515220091014670E061
:101B4000D50402D514220091F8E7150502D5132219
:101B50000091F3E7550502D512220091EEE79505B5
:101B600002D511220091E9E7D50502D51022009196
:101B7000E4E7150602D50F220091DFE7550602D5EE
:101B80000E220091DAE7950602D50D220091D5E7E5
:101B9000D50602D50C220091D0E7150702D50B22FD
:101BA0000091CBE7550702D50A220091C6E79507B9
:101BB00002D509220091C1E7D20702D00822009184
:101BC000BCE72289550702D507220091B6E79507A1
:101BD00002D506220091B1E7D20702D0052200917A
:101BE000ACE7A27AD20702D004220091A6E7A2892C
:101BF000D40603D503220091A0E719E0140702D50B
:101C0000022200919AE7540703D4940701D4D20723
:101C100002D00122009191E70020034602460146CE
:101C2000009002F017FFBDE838400248FFF746B9C0
:101C300038BD0000B40A002020070020C00A0020A0
:101C4000F0B55948594982880B889A1A92B29C2A51
:101C500064D30988818056490A880146002A0B7896
:101C600043F0020156D11646524A1C071568024637
:101C7000127822F0020274D54F4C0746E4887F7830
:101C80005FEA845C02D547F0010701E027F0010715
:101C90004770A704477802D547F0020701E027F014
:101CA00002074770670401D4E70703D0477847F07D
:101CB00008074770640603D5447844F0040404E040
:101CC0001C0603D4447824F004044470EC0450D47B
:101CD000354C9A07247824F0100423D4324D4278EE
:101CE0002F7A2D78012A45F0100514D0022A16D03B
:101CF0002D4C042AA47804F1010C0CF0FF0C13D035
:101D0000072A25D0032A23D0052A21D0062A1FD04E
:101D100021F0100142E0B90702E00570F0BD39077B
:101D20000029FADB0470F0BDFA0601D41A060AD5C0
:101D30000170022C04D280F802C0BCF1020FF2D371
:101D400041F080012AE021F0100101708670F0BDA1
:101D5000877A7F06F7D5032C04D8017080F802C07B
:101D6000F0BD0FE05107D8D51906D6D443F0800155
:101D700014E002704178CB0701D18907F0D522F039
:101D800010010BE0E9040BD49907E9D4818AC82932
:101D900002D2491C8182E3E743F00A010170DFE7C8
:101DA00002708682DCE70000F80600202007002091
:101DB00022070020B4020020C00A0020094944F68E
:101DC00048000880091D46F648000880091D41F6B4
:101DD000CC4008800348001F018841F020010180A9
:101DE00070470000182C0140084946F6680008803A
:101DF000091D0880091D41F2555008800348001F45
:101E0000018841F02001018070470000182C01403A
:101E100010B5C28800210AB1032206E002890AB186
:101E2000022202E0428912B10122027000E0017038
:101E300004784FF4804344F6206244B1012C06D06C
:101E4000022C07D0032C01D14180818010BD43803A
:101E5000828010BD41F23331418040F6B731F4E762
:101E6000401A10609168884202DA4942884200DCD8
:101E7000116051691068137E41431941936A0B4404
:101E80009362516A8B4200DD9162936A116A8B42C0
:101E900000DA9162D168936A4143107C01410341A9
:101EA000B2F91C001944884204DBB2F91A008842D6
:101EB00000DC08B270470000054920B1086940F015
:101EC00080000861704703484860034848607047D5
:101ED0000020024023016745AB89EFCD06494FF44E
:101EE0007A70CA68D20705D0401E0004000CF8D1F1
:101EF000FF20704700207047002002400E4A032058
:101F0000A2F1500182F83E00002048810B4908866A
:101F1000C862C8830884488490620948016DB1F59D
:101F2000206F01DBA3219162807A002802D0906AA1
:101F30004042906270470000640000204405002089
:101F40004C0100200449002048810881C862886251
:101F5000024988627047000064000020C008002029
:101F6000F0B53D4988894A89801A80B20F286AD322
:101F700088894881CA8939480B3A272A26D28A7823
:101F800022BB8268384B42F480728260344A374CFC
:101F9000374D12785607334A0AD4364E36881680A3
:101FA000354A12881A80354A12882280344A09E05C
:101FB000344E36881680344A12881A80334A128882
:101FC0002280334A12882A8001228A70314A0021F5
:101FD000314B82F84D1019469A7F304D0968802A9E
:101FE00032D302F01F0255F8222011422CD0826811
:101FF00022F48012184E8260123614461215B778F9
:10200000521C62F38617264AB77093F816C01778E9
:10201000BCF1800F27F0020608D30CF01F0C55F816
:102020002CC011EA0C0F01D147F0020616701A7E7F
:10203000802A0DD302F01F0255F82220114207D149
:1020400044F400218160F0BD826842F48012D1E73F
:1020500024F40021F6E7000014070020B402002059
:102060004C010020D4040020D6040020D804002015
:10207000DA040020C4040020C6040020C8040020A4
:10208000CA040020CC040020CE040020D00400208C
:10209000D2040020200D0020F4050020448F000809
:1020A000DC04002070B5204881890289891A89B230
:1020B0000F292FD3818901811C4B1D4819465D7A58
:1020C00006681C4C096846F00402802D07D305F011
:1020D0001F0554F82550294201D126F00402026060
:1020E0009A7B802A17D302F01F0254F82220114253
:1020F00011D1026822F002020260DA7A802A0ED33D
:1021000002F01F0254F82220114208D1016821F088
:102110000801016070BD026842F00202ECE701684C
:1021200041F00801F5E7000014070020F405002045
:10213000B4020020448F000830B5044600204FF45C
:102140000043024640EA030101FB01F5A54200D825
:102150000846521C5B0812B2102AF3DB30BD0000A7
:10216000F0B51D4C1B4A4FF0010C94F83B5094F80D
:102170000AE0144692F83C3094F838402B43651C32
:10218000EEB2154D95F83D700025BEF1FF0F0AD057
:10219000BEF1000F06D18B4213D155700C2C01D229
:1021A00082F83860F0BD834202D182F801C0F5E7C1
:1021B0008B42F7D15570B80709E000BF82F838505C
:1021C000F0BD8342FCD1F84382F801C080070028AB
:1021D000F4D0F0BD640400204C010020F0B5CA78B2
:1021E000002502F00F03D20601D58A7813430A783E
:1021F0004FF00F0E12F0FF0F4FF001021CD00468D9
:102200000F8802FA05F63740B74211D14FEA850C24
:102210000EFA0CF724EA070703FA0CF43C43CF78D4
:10222000282F02D0482F02D002E0466100E006616C
:102230006D1C082DE4D304600C88FF2C1ED9446863
:102240005FF0000606F1080702FA07F50F882F4035
:10225000AF420FD14FEA860C0EFA0CF7BC4303FADB
:102260000CF73C43CF78282F00D14561CF78482F19
:1022700000D10561761C082EE4D34460F0BD000057
:10228000F0B5144C002801DAE36900E06368420D00
:10229000120185B2C0F301579540C0F30346032FE6
:1022A00005D0C2020AD50322B240934307E023F0CF
:1022B0007062636823F07063636002E0AB4343F0D5
:1022C000706201B12A43002801DAE261F0BD626068
:1022D000F0BD0000000001400246002092680A4262
:1022E00000D00120704741617047016170470AB119
:1022F00001617047416170470F4A104B92F83810E6
:102300005B5C834201D1012004E00D4B5B5C8342A6
:1023100003D1002082F83A0070470A4B5B5C83428D
:1023200001D18120F6E7084B595C814201D1802020
:10233000F0E70320EEE700004C01002004930008C2
:10234000169300080A9300081C9300080A4810B569
:1023500001784FF000024C0708494FF0FF038968ED
:102360004FEA017105D5002901DA827210BD83722E
:1023700010BD0029FBDBF8E74C010020B40200206F
:10238000F0B5194E194C0022E31CA6F1060CB75CFF
:10239000A518ED78FF5C0D430F43BD421FD01CF81C
:1023A0000270FF5C0F43BD4219D015460023A618EA
:1023B000F6780E43C6545B1C1CF80220DBB2062BD9
:1023C000F5D3C17881700179C17000214218491C90
:1023D00015711CF80550C9B20629F7D3F0BD521C7F
:1023E000D2B2032AD3D3F0BDD68A000864040020F9
:1023F00010B502460021064B06205C186478944212
:1024000000D10846491CC9B20629F6D310BD000008
:102410004C010020214810B590F867100022204898
:10242000012936D11F49898899BB1F491E4B4C6C25
:1024300040F6B831B3F876308C4227DD1B49097875
:1024400021BB90F82711491CC9B280F82711C8296F
:102450001CD380F827210146D0F82C4191F828118F
:10246000A34203DD052908D2491C01E041B1491E00
:1024700080F82811C9B2052902D3012180F826115C
:10248000191B074C303CA162C0F82C31B3F5FA6F30
:1024900003D280F8262180F8282110BD200D0020CD
:1024A000B4020020EE0500204C0100201707002098
:1024B0004FF4C042C260002181620E22028241F2CA
:1024C00062024261082202834FF4604242838183A8
:1024D0004FF07842C0E9082140F6C41101807047EE
:1024E000B0F90010B0F90220891A41604269037EF8
:1024F0004A431A41836A13448362426A934200DD6D
:102500008262836A026A934200DA8262C268836AE4
:102510004A43017C0A410B41D118B0F91C208A4280
:1025200001DA10467047B0F91A008842FADC08B2A6
:102530007047000010B514481449B0F894200B8877
:102540009A1A92B2B2F5437F1DD90988A0F8941067
:10255000B0F8921020F8601F002242860C480D4C03
:10256000C2888280C180C38983812489891AA4B2E8
:10257000C4818160E11A0161074A818AC182928A1D
:102580008282511A816110BD4C0100202007002079
:10259000E80C0020440500206400002009480A4996
:1025A000B0F8B2200B889A1A92B241F684639A422C
:1025B00006D3098820F8B21F41888180002141801C
:1025C000704700004C010020200700200D480178D2
:1025D000C90702D00C49098801E04FF6FA7141663B
:1025E000094901201039088007482438018841F042
:1025F0000101018004481838018821F01801018088
:10260000704700004C010020240400400A49D1F822
:10261000982012B1521EC1F8982031F8922F521C06
:1026200021F81A294A6A521C4A628A8F521C8A87E8
:1026300001F8400C704700004C0100201CB52D48EB
:1026400090F83B3090F83C20934252D000248DF813
:10265000044053408DF800309DF800300122012BDA
:1026600008D09DF80030022B09D09DF80030042BD3
:102670000AD00DE01F498DF80420443108E01D49BF
:102680008DF80420463103E01A498DF804204831C2
:102690009DF80420012A2CD190F83D309DF800408F
:1026A000154AA34217D090F83E309DF800402342CF
:1026B00008D0B0F84C30A0F84A300B881488E31AE0
:1026C000A0F84C3090F838302BB1B0F84030148876
:1026D000E31AA0F8423012880A80A0F8402010F8CF
:1026E0003E1F9DF80020114300F801199DF80010CD
:1026F00001701CBD640400202007002070B5344D1B
:1027000040212846FFF7E8FD840080212846FFF796
:10271000E3FD44EA4004A9152846FFF7DDFD044324
:10272000E1B22C4C94F878508D4250D04D4084F852
:102730007810012D03D0022D01D0042D47D194F83B
:102740007C00A84384F87C0094F87B20AA420FD038
:1027500084F87B5094F87A2001238B401A4207D1E9
:102760001A4384F87A2094F87910491C84F8791077
:1027700094F87910042928D330B1012811D0022807
:102780000FD004280DD012E01348C18821F0400179
:10279000C1802078002184F83B1020F06000207078
:1027A00005E0217841F02001217084F83B000B49BD
:1027B00094F83B0091F82720904204D081F827003C
:1027C00007492020087000F00DF884F8545070BDBF
:1027D000001001404C010020C00A0020200D002004
:1027E0001407002070B50D4D40212846FFF774FDF9
:1027F000840080212846FFF76FFD44EA4004A915B4
:102800002846FFF769FD04430548072100F8784F83
:102810000171002141708170C17070BD00100140D4
:102820004C01002070B5344890F83A10CA43920722
:1028300061D001F0030280F8392090F83D305B064A
:102840001B0E80F83D30012A01D0812A02D15B1C89
:1028500080F83D300278D2074DD0DBB203F00102A0
:10286000C3F34004A24246D1B0F856400025641C90
:10287000A0F85640204CA0F8585090F83E60A47A3A
:10288000B24202D080F83E200DE0A607B6EB837F6F
:1028900002D080F83F5006E090F83F30642B02D21F
:1028A0005B1C80F83F3090F84030642B0CD25B1CEE
:1028B000DBB280F84030022B06D204F001039342D1
:1028C00002D1022280F84020012901D0002912D132
:1028D00090F83820416E00EB820291610163D0E9EB
:1028E00006121144D0E908231A441144826A1144A3
:1028F000C26A1144416370BD4C010020FEE7000034
:102900002DE9F04F00BF00209E4E9F4AA6F51271A0
:10291000A6F5BE79A6F1440B06F1440E804601F5FA
:10292000E074A1F1780301F5457A1D5C15F0C0074C
:1029300006D0402F51D0C02F77D0802F76D004E121
:1029400015F01F0504D0154440F080072F7201E0F8
:1029500082F80880012826D0022824D0032822D01B
:10296000042820D008281ED010281CD0874D55F8E8
:1029700020C0DCF8005054F820703D40CCF80050E6
:10298000824D55F820C0DCF8005056F820703D43C9
:10299000CCF800501D5CAD0659F820502F6813D5B7
:1029A0003AF810C03EE051F820502F6854F820C08B
:1029B00007EA0C072F6051F820502F6856F820C006
:1029C00047EA0C072F60E5E7DFF8B8C10CF1F00C1F
:1029D0005CF820C007EA0C077EE015F01F0504D064
:1029E000154440F080072F7201E082F8088001282A
:1029F0001DD002281BD0032819D0042817D008287E
:102A000015D0102813D0614D55F820502F6854F878
:102A100020C007EA0C072F605C4D55F820502F6846
:102A20005BF820C047EA0C0756E00BE056E051F88F
:102A300020502F6854F820C007EA0C072F6051F887
:102A40002050ECE715F01F0505D0154440F0800735
:102A500085F8217001E082F82180012825D0022824
:102A600023D0032821D004281FD008281DD01028E7
:102A70001BD0464D55F820C0DCF8005054F82070AB
:102A80003D40CCF80050414D55F820C0DCF80050D6
:102A90005EF820703D43CCF800501D5CAD0615D5A6
:102AA0003A4D3AF81070CC3514E051F820502F68A8
:102AB00054F820C007EA0C072F6051F820502F6807
:102AC0005EF820C047EA0C072F60E6E72D4D3AF884
:102AD0001070E03D55F820502F6036E015F01F05CE
:102AE00005D0154440F0800785F8217001E082F898
:102AF0002180012830D002282ED003282CD0042891
:102B00002AD0082828D0102826D0204D55F820C0DB
:102B1000DCF8005054F820703D40CCF800501B4DBC
:102B200055F820C0DCF80050164F883757F8207051
:102B30003D43CCF800501D5CAD06B1D4114F3AF8BE
:102B40001050E03F57F820703D60401CC0B2112883
:102B5000FFF4EBAEBDE8F08F51F820502F6854F829
:102B600020C007EA0C072F6051F820502F68DFF8CB
:102B700014C00CF1880C5CF820C047EA0C072F60E9
:102B8000D9E70000D0910008F4050020CC8F0008A0
:102B90004FF40771C1824FF45861018340F614511C
:102BA00081837047F0B5C48AB0F900608681B0F9BE
:102BB0000250C581B0F904300227002101220382AE
:102BC000AB4204DBB54202DDC78042810CE0B34278
:102BD00004DBAE4202DDC78041811CE09D4205DB83
:102BE000B34203DDC2804781018115E0B54204DBB9
:102BF0009E4202DDC280418105E0AE4205DB9D427E
:102C000003DDC1804281078106E09E4204DBAB42C6
:102C100002DDC18047810281C388458900EB4307FB
:102C200000EB4505BB89AE899B1B0FFA83FEA0F81C
:102C300012E00689AB8900EB460CBCF80CC0A3EB94
:102C40000C038382B0F91830B7F90CC0A3EB0C0C5D
:102C5000B4EB4C0F04DA80F82010A3F1A10113E0CB
:102C6000A64503DD80F82010B9890BE026B1012EBE
:102C700004D0022E10D004E0062100E0052180F8E7
:102C80002010A989091B6D31418309B2B1F5586F34
:102C900004DB5B1E438304E00421F0E7002900DC31
:102CA0004283418B8183F0BD0B49002288760A6202
:102CB000CA614A62094A32F9103002EB40028B6263
:102CC000B2F90220CA62064A32F810000882A1F85E
:102CD0006000A1F862007047040200202E930008F3
:102CE000229300082DE9F05FFE48FF4982880B8897
:102CF0009A1A92B20F2A44D30988FC4A81808346EB
:102D000011880127FA48FB4D002479B3491E118030
:102D1000C473F94A84620168B2F902204E0742F690
:102D2000AA2318D4EE8846F40056EE80F24D2D7892
:102D3000AD0709D5856825F080058560A0F87C4041
:102D400080F87E4080F87F40CD0404D480F8F07095
:102D5000C0F8EC4003E080F8F0404D0707D49A42F9
:102D600005DB80F8F470A0F8F24004E010E080F891
:102D7000F4404D0703D49A4201DBC90703D080F821
:102D80001141BDE8F09F80F81171A0F81241F8E7F9
:102D90008146B0F8181143F69820814202D2491CAE
:102DA000A9F8181101F06CFED44E96F8500010B13D
:102DB000FEF78EF905E0CB481838017821F00101C3
:102DC0000170FFF727FB00F0E5F9CD4841F26801FB
:102DD000426C4FF400608A4201DBCA4904E0B2F55C
:102DE0007A6F02DAC749091D0860B44696F85100A7
:102DF000DFF8FCA2DFF81083C44EC007AAF1300A46
:102E000036D098F80E0080282ED399F80010890744
:102E10002AD499F80F108AF80610B74950460B7853
:102E200023F002030B70AF4918394C800B7823F064
:102E300001030B70A979490611D44189B1F5FA7FD4
:102E400003D2491CAAF80A1012E040F63C718A42EB
:102E500001DD002117E108218AF8037013E1C47035
:102E60000021AAF80A400EE18AF80340AAF80A40B5
:102E7000D9F8081048460A0501D5082103E19CF855
:102E80003FE05FEACE7245D0C37B8AF8063098F8FF
:102E90000920802A4AD30278520734D4EA8892045F
:102EA00004D500BF21F02001816033E08D4A41F05C
:102EB0002001183A548092F800C02CF0010C82F8DE
:102EC00000C0816098F8171080290BD301F07F0CA7
:102ED0004FF00041D8F8002021FA0CF10A4201D14C
:102EE000077100E004710179C90702D15FEA8E71B0
:102EF00005D50321032B01D08AF80970C3E0002116
:102F0000C9F82840BFE021F020018160E98821F460
:102F10000051E98099F826014F4601280BD09CF812
:102F20006300E04648B1FDF787FF0FE0026842F01A
:102F300004020260B6E70921A5E0B968CA0502D516
:102F400021F0080101E041F00801B96097F846302E
:102F5000384642F266614FF48042D3B1012B28D04B
:102F6000022B33786A4FC3F3810333D043F6FE7CE0
:102F7000012B36D0022B34D0A0F81421A0F8442025
:102F800047F23C33A7F8003098F87030012B2BD073
:102F900038E03378C3F38103012B04D0022B02D035
:102FA00042F6146310E0A0F8141100BFA0F844200A
:102FB000EAE7337842F6CC47C3F38103012B06D00E
:102FC000022B04D043F2EB13A0F81431EEE7A0F883
:102FD0001471EBE7A0F81421A0F8442046F65473CE
:102FE000D0E7A0F814C1C9E73378C3F38103012BFC
:102FF0000FD0022B10D041F6E12300BFA0F814310E
:10300000A0F84410374918390B78DB0707D00B8A32
:1030100007E0A0F81411F3E74FF40053EEE7364948
:103020008B88ABF8123019B2B0F944305943C1F370
:103030008F335146AAF81430934200D98A82354A18
:103040001278D20605D58B8A41F23332934200D2F0
:103050008A820289C2F3C003C2F30022934205D1DF
:103060008B8A41F69912934200D98A82AA7AD207B2
:1030700000D08C82BAF81410816200297FF7E9AE83
:103080002548022104709BF81A0098B902294DD0F6
:1030900081B11B4A1078860608D5AE79760605D52B
:1030A0001C4E3678F60966F386101070E88820F416
:1030B0000260E8801248406C4E2832DBEE88300611
:1030C0002FD5BAF81220521C92B2AAF81220B2F5EB
:1030D000FA6F04D3AAF8124026F08000E880064870
:1030E00002781BE08809002020070020220700202A
:1030F000B4020020C00A0020EE050020200D0020B0
:103100004C010020100C0140F4050020DC040020DC
:1031100044010020F80600203407002022F00202BB
:1031200002708BF81A1089F80F102AE6308F0028E9
:10313000AFD143F698203087ABE770B500230C88F9
:1031400063F30F02012505FA03F6344206D0C3F1FA
:103150000F0605FA06F1114361F30F025B1C102BF9
:10316000F1DB028070BD70B500230C7863F30702B9
:10317000012505FA03F6344206D0C3F1070605FA25
:1031800006F1114361F307025B1C082BF1DB0270AF
:1031900070BD0000F0B51F4890F866301E48012B46
:1031A000816821F4006232D11C4BDE8874062ED473
:1031B0001B4D0F054FF00004B5F902501ED4194AFB
:1031C000526C642A11DC40F6386295420DDAB20482
:1031D0000BD4027852070ED4B0F8D42040F6B8359C
:1031E000AA4203D2521CA0F8D420F0BD41F40061E1
:1031F00081605C81F0BDA0F8D440F0BD41F2CD010A
:103200008D42FADD997AC907F7D18260F3E78260CF
:10321000F0BD0000200D0020B4020020C00A0020F4
:10322000EE0500204C010020F0B5364D364F044627
:1032300095F83B0097F83B1023780843EE1C627822
:10324000834205D1E0781146FEF78AFF207908E035
:1032500094F802C084450CD1E1781046FEF780FF57
:10326000E07905F82F0F2878805D6870287BE87773
:10327000F0BD82421DD161461846FEF771FF95F8F8
:103280004E1095F83B00814207D1B97A09B1A17976
:1032900000E0617985F82F101EE06978012901D0DE
:1032A000A17922E0617927E0297841F004012970B1
:1032B00012E0E1788142DBD119466046FEF750FF0B
:1032C00095F84E1095F83B0081420AD1B97A09B1C0
:1032D000617ADFE7217ADDE715F82F1F895D6970D4
:1032E000C5E76978012906D0617A85F82F10B97A87
:1032F0000029F1D1D8E7217A85F82F10B97A002971
:10330000EAD0D1E7640400204C0100200B4801788A
:1033100021F0020100F8381B002100F8181941774C
:10332000817733218185418508214184012100F87D
:103330001F1C034880F83910704700006404002007
:103340004C0100200D4900B50B4851F8012F40F801
:10335000032F89888180084801210930FFF710F880
:10336000054802211330FFF70BF8034804211D30F4
:103370005DF804EBFFF704B8640400204C01002062
:10338000094944F648000880091D46F648000880AF
:10339000091D41F2111008800348001F018841F007
:1033A0002001018070470000182C01402DE9F047F2
:1033B000664C674B0025A0780126654A1033052826
:1033C0007ED2DFE800F00313113E1100108820F0D8
:1033D000010010801D805F480580001F0580001FD0
:1033E0000580FFF7CDFFA670BDE8F087594941F28F
:1033F00044401C390880574945F658002439088054
:10340000091D47F2580008805249202028390880B9
:103410000020401CC0B27328FBD3FFF7B1FF4C491A
:1034200084F85C502C3147F690600880484814308E
:1034300006801D80108840F0010010800220A070DE
:10344000D2E700215FF0010004EB410204EB4003EE
:10345000B2F85020B3F850309A4200D20146401CD6
:10346000C0B20628F0D33C48405C84F83900FFF72E
:103470004DFF1D2000F0F3F900F076F8374E384884
:103480004FF4807996F83B10012904D002291BD013
:10349000042930D047E040218046FEF71DFF870019
:1034A00080214046FEF718FF47EA4007494640465C
:1034B000FEF712FF074347F0010084F83B0000E0ED
:1034C0003DE0224809302CE040218046FEF704FF11
:1034D000870080214046FEF7FFFE47EA4007494645
:1034E0004046FEF7F9FE074347F0020084F83B0030
:1034F0001648133015E040218046FEF7EDFE8700A8
:1035000080214046FEF7E8FE47EA4007494640462C
:10351000FEF7E2FE074347F0040084F83B000B4847
:103520001D3002F07FFE94F82F0086F838001D2031
:1035300000F0ABF90420A0700A48057054E7108829
:1035400020F0010010801D80A5704DE7640400206C
:10355000000800403C2C0140DC8A00084C0100209F
:1035600000100140170700202DE9F041344C14F8F9
:103570002F0F344DE07240212846FEF7ADFE860045
:1035800080212846FEF7A8FE46EA4006AF153946D8
:103590002846FEF7A1FE0643207BF1B22F3C814274
:1035A00015D084F83C0040212846FEF795FE8600A1
:1035B00080212846FEF790FE46EA40063946284616
:1035C000FEF78AFE064384F83B60FFF737F81E4D8E
:1035D00095F83B00012827D0022828D0042829D0BC
:1035E000174894F83B102730085C04F8300F14F8A3
:1035F0000109FEF7FDFE04F82F09A87A00B10120A9
:10360000607001F0DBFA94F84E0094F83B108842A9
:1036100006D094F83800062802D2401C84F83800FE
:1036200084F84E10BDE8F0810548093004E00448F4
:10363000133001E002481D30BDE8F041FFF7F4BD52
:1036400064040020001001404C0100202DE9F041ED
:10365000524991F87200AA287CD191F8730055283C
:1036600078D14F4C00200A5C2254401CC0B2742810
:10367000F9D34C4E2069C6F80100A08AA6F80500CF
:10368000D4F81600F060D4F81A003061D4F81E00A7
:103690001234706102F06CFD4349608A888102F047
:1036A00081FD207D123CC007307802D040F004003C
:1036B00001E020F004003D4930704FF480403C4D63
:1036C000886114F8280F85F82000608B6880A08B33
:1036D000A880E08BE880208C2881608C354F688141
:1036E00094F8240087F8D20014F8011C304686F8BC
:1036F0003B100026C0F89C60FFF724FE2E48A18EE8
:103700000183E18E4183218F818394F84210283C0C
:10371000012908D0022901D0032909D0297821F0F4
:103720000C01083107E0297821F00C01091D02E0A5
:10373000297841F00C01297094F86E1059B10122DA
:10374000012901D0022909D087F8462094F8641095
:1037500051B907E016E087F84660F7E7022187F8DD
:103760004610F3E715494E8194F8701001290BD0EB
:1037700094F86D1059B101290CD04FF4805100BF5D
:10378000A0F87610BDE8F08144F21C71F8E74FF420
:103790000051F5E741F25551F2E7000000FC000846
:1037A000200D00204C01002064000020B80C0020F7
:1037B000DC040020B402002044050020C00A0020E0
:1037C0007CB50121082000F089FB4FF48070ADF832
:1037D000040010248DF8074001208DF8060001A98F
:1037E0001548FEF7FBFC0121092000F077FB0121C1
:1037F0001248FEF745FD0820ADF8000004208DF8C2
:1038000003000F4E03258DF8025069463046FEF73F
:10381000E5FC08213046FEF766FDADF800408DF866
:1038200003408DF8025069463046FEF7D7FC102160
:103830003046FEF758FD7CBD001401400002300008
:10384000000C0140FEE7704700F01F02012191408B
:103850004009800000F1E020C0F88011704700F0BE
:103860001F02012191404009800000F1E020C0F8D2
:103870008011704700F01F02012191404009800033
:1038800000F1E020C0F80011704700F01F02012194
:1038900091404009800000F1E020C0F8001170471D
:1038A00070B50F23C47801780122F4B1144C246858
:1038B000457804F4E064C4F5E064240AC4F1040625
:1038C000E3408478B5401C402C4301F1E021230102
:1038D00081F80034007800F01F018A404009800020
:1038E00000F1E020C0F8002170BD01F01F0082400F
:1038F0004809800000F1E020C0F8802170BD000080
:103900000CED00E0024908430249086070470000DE
:103910000000FA050CED00E02DE9F05F00261D2007
:10392000FFF792FF6C4CDFF8B4B1A4F1B800A77EAA
:1039300090F83810DFF8A8E1DFF8A8A100258F4241
:103940007ED0E776A176626A036B5A434FEA12494A
:103950009BF80820120702D51EF8012000E00A4655
:1039600094F812C0BCF1010F09D004EB4206B6F97D
:1039700002C0C4F828C0B6F90460E6620CE043F661
:10398000FF7CC4E90A5C90F83DC05FEACC7C01D0C2
:1039900012B102E0052A00D1012600EB47074FF0E3
:1039A000804CBF893F04B7FBF3F3E361476BBCFB7B
:1039B000F7F7276294F813C0BCF1000F06D0BCF1F2
:1039C000010F05D03B4403EBD3735B10636201E04E
:1039D0003B466762DFF810C14FF6FF7707EA8307BF
:1039E000ACF808709AF8007090F80A8090F83DC022
:1039F000082F08F003070CF0030C05D067450BD126
:103A0000B8F1000F05D008E0674505D0B8F1000F08
:103A100003D05B42636200E06562C6B1636A002B5B
:103A200003D006DD228D05E00AE0304B33F812208A
:103A300000E0A28DA4F86020227822F020022270FB
:103A40009AF80020042A07D0082A05D012E0B4F81A
:103A5000603003EB0902EDE780F8405065629BF8A7
:103A60000800000701D51EF80110204830F81100A9
:103A7000A4F860001E49606A09883E314843B4F8E2
:103A8000601001EB204006B21D20FFF7F3FE606AD4
:103A9000002807D021784FEA81600ADD002804DA87
:103AA000A08D09E0B4F8600006E0E06AB04208DBEF
:103AB0000CE0002802DA208D208208E0A06AB042E3
:103AC00004DD208241F02000207000E02682257570
:103AD00065752586BDE8F09F04020020B402002031
:103AE0001093000817070020540A002022930008B2
:103AF0002404004043184FF48042934210DD90426A
:103B000002DD104600210BE0914202DD002011464B
:103B100006E08003B0FBF3F000B2C0F5804109B2CB
:103B200041EA00407047F0B541F2B8430022C3605B
:103B30000E248262048249F27E15082645610683BE
:103B400043F6FF774283878340F2492E4FEA873C52
:103B5000C0F808E0C0E9082CCB608A620C824D6195
:103B60000E834A838F83B4208860C1E9082CF0BD9E
:103B7000002181620949C1600E2101820849416129
:103B8000082101834FF44041418343F6FF71818353
:103B900009070162034941627047000095890200EC
:103BA000F0A1010000C0FF0F064941F6A2600880A5
:103BB00005480168054A01F4E06111430160BFF363
:103BC0004F8FFEE7442C01400CED00E00400FA05A5
:103BD00038B501210D2000F081F94FF4E060ADF817
:103BE000000018248DF8034003258DF80250694623
:103BF0000D48FEF7F3FA4FF46040ADF800008DF881
:103C000003400A4C8DF8025069462046FEF7E6FA5A
:103C1000A014ADF8000048208DF803006946204646
:103C2000FEF7DCFA38BD000000080140000C01403E
:103C30002DE9F0410121CE028CB0304600F04EF962
:103C4000DFF86C81404601F02DFC08A801F056FE1B
:103C50004FF45860ADF824000024ADF82040202037
:103C6000ADF822000125ADF826408DF8285008A9AE
:103C7000404601F0F5FD0021404601F048FE4FF6B8
:103C8000FF71404601F04DFE01220021404601F047
:103C9000D9FD0121404601F0C1FB04A801F0D9FB88
:103CA000ADF81060A802ADF81200ADF81440A220E3
:103CB000ADF816002803ADF81800ADF81A40ADF8BD
:103CC0001C4004A9404601F0B3FB6027ADF800702A
:103CD000ADF80440ADF80840ADF80C40ADF8024036
:103CE000ADF80640ADF80A40ADF80E4069464046D2
:103CF00001F098FC6946404601F0DAFC694640460E
:103D000001F020FDADF8045040F61450ADF80070FD
:103D1000ADF80600ADF80840ADF80C40ADF8025023
:103D2000ADF80A40ADF80E406946404601F04EFD40
:103D30000121404601F096FB0821404601F0B2FC0B
:103D40003146404601F0F4FC0821404601F038FDC0
:103D50003146404601F06CFD7021404601F075FD92
:103D600018208DF82C008DF82D408DF82E408DF800
:103D70002F500BA8FFF794FD0D480C30018841F03F
:103D8000800101800A481430018841F0010101805E
:103D9000001F04800121404601F06EFB8DF8285081
:103DA0000121404601F072FB0CB0BDE8F08100003B
:103DB000002C0140704740F21341416008218160AE
:103DC0008621C1604FF48041016149424161002177
:103DD0000162C162704701627047000010B501883E
:103DE0004288891A09B20183B1F5005F02DBA1F5AF
:103DF000804104E011F5005F02DC01F580410183A0
:103E0000B0F9182041685143C1618368846A534303
:103E1000C2681B12624303EB2222036A1A44114454
:103E200002628A13426241698A4203DB01698A4263
:103E300000DC11468A1AC0E90A21028E4FF403738E
:103E4000594302EBA13202860B4A1278082A04D1A8
:103E50000A4A936F03EBA1319167B0F93010B1F5C5
:103E6000804F02DDA1F5804103E0002902DA01F56F
:103E70008041018610BD000017070020D40A0020F1
:103E8000034A516821F440410143516070470000EA
:103E900000100240044A0029516901D0014300E0AA
:103EA000814351617047000000100240044A00291C
:103EB000D16901D0014300E08143D1617047000026
:103EC00000100240044A0029116901D0014300E0BA
:103ED000814311617047000000100240044A00292C
:103EE000916901D0014300E0814391617047000076
:103EF00000100240044A0029D16801D0014300E0CB
:103F00008143D160704700000010024030B5244961
:103F10004A6812F00C03234A03D0042B01D0082B6B
:103F200026D002604A680F231F4C03EA1212A35CDA
:103F30000268DA4042604B68072505EA1323E35C18
:103F400022FA03F383604B6805EAD323E35CDA408B
:103F5000C2604B68032403F4404104EA933303EB4B
:103F60009161114B1B1F595CB2FBF1F1016130BD36
:103F70004A680E4B1A404B68140103F4803303D592
:103F8000C2F38342113202E0022404EB924213B1E5
:103F90004B689B0301D5064B00E0024B5A43C0E738
:103FA0000010024000127A000400002000003C08CB
:103FB00000093D002DE9F041274CA615402120467F
:103FC000FEF78AF9850080212046FEF785F945EA4B
:103FD000400531462046FEF77FF90543EDB240210A
:103FE0002046FEF779F9870080212046FEF774F914
:103FF00047EA400731462046FEF76EF90743F8B21C
:10400000A842DBD140212046FEF766F987008021D7
:104010002046FEF761F947EA400731462046FEF7A1
:104020005BF90743F8B2A842C8D140212046FEF709
:1040300053F9870080212046FEF74EF947EA4007F2
:1040400031462046FEF748F90743F8B2A842B5D1F9
:104050002846BDE8F08100000010014010B502685C
:10406000416802FB02F301FB0133B3F1805F11D918
:104070001B0E103B0A4C9BB212B234F8133009B23B
:104080005A43594342F38F3241F38F31C0E9022141
:10409000012102E0C0E902210021017410BD0000ED
:1040A000908A00082DE9F05FF848F94902880B88EA
:1040B0009A1A92B20F2A7DD309880180F5480246E8
:1040C0008189D2884B0703D48B0701D4CB0702D058
:1040D00042F4007201E022F40072C28081460807B7
:1040E00002D44846C90604D5B9F8061041F00101CA
:1040F00002E0C18821F00101A9F80610E548FDF7AA
:1041000087FEE5484FF4804BB0F93A10594502DA82
:10411000491C418702E0E049A1F83AB0DFF87C830E
:1041200041F6CC40DE49D8F85020824203DD886851
:1041300020F010008860DB4BDB4E0024188820B193
:10414000401E1880CC73347027E0B9F8060045048F
:104150001BD4B9F80C30DD0617D41B0715D40306A1
:1041600013D4830611D403050FD4430603D5CF4BD4
:104170001B781B0609D5430707D4C30505D40307DD
:1041800003D4830401D4C00607D5C948CC73C94BF6
:104190003470C4831C8080F828408A460846C98F42
:1041A000DFF814E359B1491EC187C4490B7823F0E5
:1041B000020300E0EEE00B708AF80F400BE0BF480E
:1041C000017841F0020101703078012804D19EF895
:1041D0000000062800D134703078B94D01270A2834
:1041E00072D2DFE800F0FCD705D7FBFAD771F9F8F7
:1041F00002F0D4F8DFF8A892A848A9F13009B9F87C
:104200001810491C8AB2A9F81820416C40F62820E1
:10421000814202DAA9F8184014E09F4840F6CC43E6
:10422000C06898420EDBA54843F69913B0F9040024
:10423000984207DBB2F5FA7F04D32A7812B9A9F8BD
:1042400018402F709F4A108868B199F804305B1CA1
:10425000DBB289F80430022B05D39B4889F804406F
:1042600003885B1C03809AF80F00D046092812D0FF
:1042700002287DD0A8F83041B8F84000A246C8B165
:1042800041F288345046A9F818A0A14221DA2978D1
:1042900001291AD01DE07D484430FEF709F9FDF7E9
:1042A0002DFE7E48416CC9F82C1041F27C51C9F8B2
:1042B0001C105CE2A88AA8F83000E86A6863A86A63
:1042C0002863A8F8407037E0A1E17F492870088092
:1042D00010807E4940F63A2291F8681001290DD0ED
:1042E000C8F8D80088F8EA00C9F82400B8F93010F6
:1042F00001F21D50904218D8102317E098F82811A9
:1043000001B97348C8F8D80088F8EA70B8F93010D5
:1043100001F21D509042B8F8D80000B202D8102324
:104320001A4605E02023022202E02023102200206A
:1043300000F09CFBA8F83000644866494FF4F07325
:1043400090F868000128554815D0406C40F2DC52C6
:10435000904203DAB5F90A209A4215DDB8F84020F8
:1043600040F6C413521C92B2A8F840209A4200E0D2
:104370001BE009D210E0426C40F2DC50824209DAC4
:10438000B5F90A00984205DC86F800A088F8EAA092
:10439000A1F81AA0BDE8F09F3F4AD268002AF9DCD4
:1043A00042F6E0629042EFDAF4E7B8F8300140F606
:1043B000B832904207D2354B183B1B78DB0702D14D
:1043C000401CA8F8300183B240F2DC50834207D889
:1043D00042F6CC4008E0B0E08EE0D5E0D0E0D8E096
:1043E000A8F8302143F26660E867C9F82C1089F814
:1043F0000870394EA8F8404088F8EA40707F4D4672
:10440000F0B1F07F80B3B8F82800B8F9301000B2EE
:104410000A23052200F02AFBA8F83000F47774770D
:10442000B8F91601B8F91411884229DA697901F14D
:10443000010111F0FF01697152D06C71401C21E043
:10444000A8F8E4B0D8F828105846814200DA0846A7
:104450001E4900B2E88291F84D100029B8F93010D9
:1044600003D03623052203E005E040F2471336224D
:1044700000F0FCFA01E040F26660A8F83000CFE7F7
:104480002CDD801EA8F816012AE000008809002013
:1044900020070020C00A0020440500204C01002015
:1044A000B40200202407002017070020F80600208F
:1044B000F00800201E00002018070020EE05002054
:1044C000640000202000002022000020200D002099
:1044D0009AF9FFFFFC090020E80C0020A8F816114B
:1044E000B8F93000584502DDA8F830B052E700288E
:1044F000FCDAA8F830404DE7D149DAF8DC20504624
:104500008A4202D2521CC0F8DC20C27B082A03D1A6
:10451000D0F8DC208A420CD334708168CA0502D5F9
:1045200021F0080101E041F008018160CAF8DC4097
:1045300030E7BDE8F05F02F09FBC9AF80F005746E5
:10454000092803D03C868AF80F404FE1BD4D286A08
:10455000401C2862022809DDA88D012301B2A88B26
:10456000052200B200F082FA2C62E862B648A98DFA
:104570000180B8F844104180FDF7B2FF388609E7A2
:10458000BDE8F05F04F046B9B048007809287DD056
:1045900000E78AF80D419AF8281161B142F3110041
:1045A000CAF8D840AA498203E86280108A6281036F
:1045B000A862A8488162A3480483D8F8441041F255
:1045C0008830814207DA2878012804D1A2482C706B
:1045D0000480A2480480A249A24B0888401C82B2F1
:1045E000A1480A80C82A04D390F800C0BCF1010F8A
:1045F00019D0B2F57A7F04D390F800C0BCF1020F55
:1046000011D0B2F5FA6F02D30278032A0BD09AF8D0
:104610000F00801E082873D2DFE800F00FABEAFE1F
:104620000472739DB6E604700C80B9F8061021F48C
:104630000061A9F806101F70E9E7FDF787FE98F8FA
:104640000000400613D58948807804280FD0D8F898
:104650004410404682290ADA817A98F83D0001F038
:10466000030100F00300814201D001F047FD3078E2
:10467000B14606288CD088F83F40D8F8500046460E
:1046800040F3110082037249E86200E0AEE080105E
:104690008A628103A8626F488162FDF72FFC694836
:1046A00055460772BAF81401AAF81601706CAAF8F8
:1046B0008240B0F5437FAAF880B00CDDA86840F4D2
:1046C0008060A86096F838100529ABD140F0100042
:1046D000CAF8080010E0A96821F48061A96040F2DE
:1046E0008A21884204DA3078400601D402F0B0FA18
:1046F000A86840F01000A860022089F8000049E690
:1047000095E0D8F84400B0F5437F06DA9EF8001033
:10471000062902D08EF8004082E05548017821F049
:1047200040010170FDF7EAFB43F6FE70AAF816019E
:104730000AF1DC05FDF70AFE4E4810F8341F21F09F
:104740000101017043492C608C6241498C6208214F
:10475000317044641EE63C48FDF7AAFEFDF7CEFB2F
:104760003848D8F84410C16241F27C51C161092037
:104770003AE099F80600C006C1D4D8F8440045468E
:10478000B0F57A7F32DDFDF7E1FD2878400611D5DE
:104790003648807804280DD0686C82280ADAA87A16
:1047A00095F83D1000F0030001F00301884201D0AC
:1047B00001F0A4FC85F83F40B5F85000AAF830009D
:1047C00001B25446594501DDA4F830B0FDF796FB1F
:1047D000A06840F48060A06095F8381005298ED15B
:1047E00040F01000A06002203070D3E53470D1E5B5
:1047F000D8F84400B0F5437F03DA9EF8001006298C
:1048000088D1B9F8061021F02001A9F80610FDF7AB
:104810009DFD0420E8E7FFE79EF80000062801D090
:104820003770B7E50949092008700520DCE70F4813
:1048300084708EF8004085F85E40AAF83040A9E503
:10484000C0D4010084020020CC0900206C020020AA
:10485000C008002090080020220000202000002036
:104860001600002014000020150000206404002021
:1048700026070020D40A002030B585B0012104208D
:10488000FFF72CFB4FF40040ADF8100048208DF8E6
:10489000130004A91848FDF7A1FC01210846FFF701
:1048A00005FB40F68C20ADF8040003240020ADF891
:1048B0000040ADF80200ADF806004FF080456946B3
:1048C000284600F0CDFF1C208DF80C008DF80D401F
:1048D0008DF80E4001208DF80F0003A8FEF7E0FFD1
:1048E00001221146284600F095FE0121284600F0DD
:1048F000C3FD05B030BD0000000801407047000056
:104900002DE9F041304CE07800285AD12078002879
:1049100057D0401E10F0FF00207052D14FF4967017
:10492000208272B6294F45F2AA50A7F872000020E3
:10493000FDF7C2FA264D13202860FDF7CFFAA8BB79
:104940003420E86002202861224E6E61286940F020
:1049500040002861FDF7C2FA40BB00211E4A08460C
:104960005FEA255312F800C0BCF1FF0F00D001210F
:10497000401C80B29842F5D3C1B9C4E90676392605
:104980000127A06910F8011B10F8012BA061E06954
:1049900001EB022102886A612F6120F8021BE061AD
:1049A000FDF79CFA10B9761EB6B2EAD20120FDF7E7
:1049B00083FA62B601F0F6FB0848816821F4804171
:1049C0008160BDE8F081000014070020200D002068
:1049D0000020024000FC000800FC0008B402002097
:1049E0001948016841F010010160016821F00301DC
:1049F0000160016841F002010160144841684160B2
:104A000041684160416841F480614160416821F43E
:104A10007C11416041680E4A11434160016841F0D8
:104A20008071016001688901FCD5416821F00301B2
:104A30004160416841F0020141604168C1F3810178
:104A40000229FAD170470000002002400010024005
:104A50000000280830B5044C039D6080A180E280EE
:104A60002381658130BD0000B40A00200A448242DF
:104A700001DA10B27047C91A8142FBDD08B27047F3
:104A80002DE9F0434648DFF81C91DFF81C81C17F17
:104A9000467A04680022454B4548802930D301F00E
:104AA0001F0559F825100C420146096802D041F44F
:104AB000805101E021F480510160CD041CD48D04AB
:104AC0001AD59D7AED0707D05A8198F8005025F045
:104AD000020588F800500FE090F846500127DDB13C
:104AE0004FF0020C012D1CD00327022D1CD080F8A2
:104AF000462000BF80F81A710D0B65F34D3101603F
:104B0000802E2DD306F01F0559F825100C420168A0
:104B10000FD041F004010EE080F8467080F81A21B1
:104B2000EAE780F846C0E5E780F8467080F81AC1E9
:104B3000E2E721F0040101604C070DD44C050BD5D0
:104B40009C7AE40708D05A8198F8004024F00204C7
:104B500088F80040C0F898208C0864F38A2101602E
:104B6000997AC90716D1134991F86410012911D116
:104B70001149496C32290BDC0178490708D50189B4
:104B8000090505D4D0F8981047F23053994203D95B
:104B9000C0F89820BDE8F083491CC0F89810F9E7E8
:104BA000F4050020448F0008EE050020C00A002014
:104BB000B4020020200D00204C01002010B5FCF7AD
:104BC000D1F80F48018821F0020101800C49183109
:104BD00009880C4A928E1144094A343211800849DE
:104BE0000C390A8842F001020A80011D0A884FF63A
:104BF000ED531A400A80018841F01201018010BD76
:104C00000C0400406404002006484188491C89B215
:104C10004180B1F57A7F04D38188491C81800021CD
:104C200041807047380700200F4810B5016841F0F7
:104C30000101016041680D4A1140416001680C4A60
:104C400011400160016821F480210160416821F474
:104C5000FE0141604FF41F018160FFF7C1FE05496D
:104C60004FF00060086010BD001002400000FFF827
:104C7000FFFFF6FE08ED00E02DE9F0413149324D2D
:104C80000888401C088028884FF00004000629D5B9
:104C9000FCF7F4F92D4A2E4807231778C8262D492A
:104CA000012F22D02C4FB7F806C0BCF1000F3ED028
:104CB000B0F80CC04CF0080CA0F80CC0B0F806C05E
:104CC0002CF4006CA0F806C0886820F0040088600E
:104CD000FC801370CE8700204FF49661401C80B298
:104CE0008842FBD32C80BDE8F0811C4F97F800C0B0
:104CF000BCF1010F0FD0BCF1020F11D0B0F806C00B
:104D00004CF4006CA0F806C0886840F0040088608D
:104D100005203870DDE7B0F80CC04CF0080C03E05B
:104D2000B0F80CC04CF0100CA0F80CC0F0E70C4F21
:104D30003C70C78847F40067C780886840F004006B
:104D40008860C6E738070020102C014017070020B4
:104D5000C00A0020B40200208809002018070020A3
:104D600035070020704700002DE9F0434FF08040E8
:104D7000018A21F001010182AA48007800287CD133
:104D8000A94FF87B002878D1A848406C322874DC01
:104D9000A7488068DFF89C924104A74DB9F8040049
:104DA0004FF0000403D4401CA9F8040024E10028BB
:104DB00074D02978012611B1012912D013E1494696
:104DC000B0F5BE7FFAD92E70CC718C71EC702C725C
:104DD000287A0A18401CC0B2147228720F28F7D320
:104DE00001E1B9F802204946824201D9EE7100E0A2
:104DF000EC7190488A7908300F2A15D2CB79082BAC
:104E00000BD2C3F10708EB7912F800C003FA08F3DC
:104E100063441354CA79521CCA71CA79082A03D14F
:104E20008A79521C8A71CC7199F80610C8460F29EC
:104E300073D10D21FCF78CF8A881010A6970C0B20A
:104E4000A87088F8064098F816208A4265D198F82C
:104E50001510814261D198F80BC0784903230222D2
:104E60007748BCF1000F10D0BCF1010F02D0BCF1AB
:104E7000020F14D080F86A2000E0C7E091F800C06B
:104E80002CF00C0C0CF1080C0FE080F86A6091F823
:104E900000C02CF00C0C0CF1040C06E0A5E080F82E
:104EA0006A3091F800C04CF00C0C81F800C098F802
:104EB0000C10B6EB111F04D180F86E4087F8464005
:104EC0000EE0B2EB111F04D180F86E6087F84660E7
:104ED00006E0B3EB111F03D180F86E2087F846205F
:104EE0000B0717D001F00F01012901D0022915D0BD
:104EF00080F86C602C7198F80D102A7906FA02F38C
:104F00000B406B71082A41D2DFE802F00B0F40160C
:104F1000212C333A80F86C40ECE764E080F86C2098
:104F2000E8E713B380F8704030E013B180F85060C8
:104F30002CE080F8504029E023B180F8656087F8C4
:104F4000036123E080F8654087F803411EE023B148
:104F500087F8F54080F84D4018E087F8F56080F854
:104F60004D6013E013B180F868600FE080F868408E
:104F70000CE013B180F8666008E080F8664005E058
:104F800013B180F8676001E080F86740521CD2B22C
:104F90002A71082AB1D398F80E108A0704D587F829
:104FA000F16080F8646005E0264A87F8F14080F8F7
:104FB00064405481C90702D080F8294001E080F89C
:104FC000296098F8111000F86D1FC2781E48012A58
:104FD0001ED001B3012921D04FF48051A0F87610E2
:104FE0001A493C200870A9F80240A9F80440B9F811
:104FF0000210491CA9F80210B9F80210B1F5FA7FA5
:1050000004D940F2F511A9F802102C70BDE8F08324
:1050100044F21C71E2E74FF40051DFE741F25551D1
:10502000DCE7000017070020B40200204C0100203C
:1050300000100140080D0020B0060020DC04002014
:10504000200D0020C00A0020440500201407002085
:105050002DE9F05FFDF77AF98E4D2888A5F1040659
:10506000C0070AD0308820F008003080288820F05F
:105070000900288001F0ECFDD9E02888DFF81892BB
:10508000DFF81882864C80071AD5B9F8001041F075
:105090000101A9F80010B8F800008049143150301F
:1050A000088028884FF6F95108402880308840F061
:1050B00004003080FEF77EFF84F83C00BDE8F09FDE
:1050C0002888784F4007288871D520F00400288070
:1050D000FEF770FF94F83C108142EFD1308820F049
:1050E00004003080FDF70AFB2078410605D594F8CE
:1050F000541094F83B209142E0D03978400621F0DA
:105100000201397004D5FEF72FFA97F82F7004E0EA
:1051100094F83C00FDF76CF90746DFF880B140F6E3
:105120008C2A0BF1180B062F47D294F83800B8429E
:105130003ED03846FDF7E0F82078C00716D094F846
:105140003A0094F8391000F00302914206D0A17A97
:1051500000F0010001F00101884215D1FDF736FA97
:10516000FBF74CFEFDF75EFB384689E0FDF72EFAB3
:10517000FBF744FEFDF756FB3846FDF747FA20786B
:1051800040F00100207099E7288820F0080028806E
:10519000206B810801EBD000504515D2B8F8001003
:1051A0000844ABF80000308840F0080003E00DE050
:1051B000308820F00800308080E7B9F8001041F016
:1051C0000101A9F80010DFE75046E7E7000728884B
:1051D00031D520F008002880308820F00800308089
:1051E000FEF7E8FE84F83C00FDF788FA387820F0F6
:1051F000020038702078400604D5FEF7B5F997F81C
:105200002F5004E094F83C00FDF7F2F80546062D17
:1052100008D294F83800A842B5D0FDF7D7F9FBF7CB
:10522000EDFD2AE02048C18841F04001C180BDE881
:10523000F05FFDF7D7BAC006288825D520F010000A
:105240002880308820F01000308097F838000C2833
:1052500002D2401C87F83800387840F002003870DD
:10526000FEF782F997F82F50787884F8390094F88F
:105270003800A84287D0FDF7A9F9FDF7D3FA2846F0
:10528000BDE8F05FFDF7C2B94EF2BE1108402880BC
:1052900014E7000010040040000400402404004013
:1052A0004C01002064040020C00A00202DE9F04FCA
:1052B000514F85B0388820F0010038804E480026D4
:1052C000103006804D4CDFF838A14FF0010894F8FB
:1052D0005C0042F63029C10774D072B64948816932
:1052E00041F400718161816941F4806181614FF411
:1052F0000040FEF7C5FD444D00212846FBF7DCFACF
:1053000000212846FBF7CEFADFF800B1002158460D
:10531000FBF7C8FA00213E48FCF732F92846FBF7B4
:10532000E7FB5846FBF7E4FB4FF46020CDE90206AB
:105330008DF8056000968DF810808DF80480694620
:105340002846FBF767FC01231A460F212846FBF786
:10535000B2FC01212846FBF7A5FA00204946401C73
:1053600080B28842FBD328462E600121FBF7E2FC85
:1053700028688007FCD524484C30006894F85C10FD
:1053800021F001012144A1F85000FBF79FFA62B619
:10539000FDF7F6FF47F69061AAF8001094F85C005C
:1053A000401CC0B284F85C000C2822D2124914318F
:1053B000A1F80080388840F00100388005B0BDE8D1
:1053C000F08FFFE7134920F00100085A12490880C6
:1053D000114945F65800083908800F4847F258012E
:1053E000001F01800C4920200C390880AAF8009089
:1053F000D4E70320A070E1E7000800406404002027
:105400002C08004000100240002401400028014008
:1054100008000240008B0008202C01400029018870
:1054200002D041F0800101E021F08001018070474D
:1054300010B50A884B88CC881A438B8823431A43BB
:105440000B891A434B8989891A430A43A0F84420DF
:1054500010BD0021018041808180C1800181418196
:10546000818170470029818802D041F0010101E06B
:1054700021F00101818070470029018802D041F0AC
:10548000010101E021F0010101807047002930F89D
:10549000441F02D041F4004101E0C1F30E0101803C
:1054A000704700004B4910B5884202D10121C41455
:1054B00086E0B0F1804F09D0474988420DD10121E3
:1054C0000220FEF7FFFC0021022064E001210846D3
:1054D000FEF7F8FC002101205DE04049884206D13A
:1054E00001210420FEF7EEFC0021042053E03C499A
:1054F000884206D101210820FEF7E4FC00210820A3
:1055000049E03849884206D101211020FEF7DAFC33
:10551000002110203FE03449884206D1012120209B
:10552000FEF7D0FC0021202035E03049884202D12E
:105530000121441444E02E49884202D10121CC04C7
:105540003EE02C49884202D101210C0538E02A496D
:10555000884202D101214C0532E02849884206D117
:1055600001214020FEF7AEFC0021402013E0244939
:10557000884206D101218020FEF7A4FC0021802072
:1055800009E0204988420AD1841501212046FEF70E
:1055900099FC00212046BDE81040FEF793BC1A4953
:1055A000884202D101210C040AE01849884202D144
:1055B00001214C0404E0164988420AD101218C04DF
:1055C0002046FEF797FC2046BDE810400021FEF77C
:1055D00091BC10BD002C01400004004000080040B8
:1055E000000C004000100040001400400034014056
:1055F000004C0140005001400054014000180040A0
:10560000001C0040002000400040014000440140D8
:1056100000480140002A828901D00A4300E08A4301
:105620008281704730B5028C22F001020284028C24
:105630008388048B22F0020224F073050C882C432B
:105640000D8915434A882A43114DA8420BD0114DAC
:10565000A84208D0104DA84205D0104DA84202D053
:105660000F4DA8420DD122F008054A8923F440735A
:105670002A4322F004058A882A438D891D43CB8959
:105680002B4383800483C9888186028430BD000057
:10569000002C014000340140004001400044014022
:1056A00000480140028B22F008020A43028370473F
:1056B00070B5028C22F010020284028C8488038B65
:1056C0000D8823F4E6464FF6FF7303EA05253543BC
:1056D0000E8922F0200203EA061616434A8803EADE
:1056E00002123243104EB04202D0104EB04215D1D9
:1056F00022F080064A8924F4406403EA021232430D
:1057000022F040068A8803EA021232438E8903EAB5
:1057100086062643CC8903EA8404344384800583C7
:10572000C9880187028470BD002C0140003401400B
:10573000028B4FF6FF7322F4006203EA012111434A
:105740000183704770B5028C22F480720284028C4F
:105750008488838B0D8823F073031D4322F4007328
:105760000E894FF6FF7202EA06261E434B8802EAB4
:1057700003233343104EB04202D0104EB04215D135
:1057800023F400664B8924F4405402EA0323334394
:1057900023F480668B8802EA032333438E8902EA6E
:1057A00006162643CC8902EA041434438480858398
:1057B000C9888187038470BD002C014000340140FA
:1057C000828B22F008020A438283704770B5028CF4
:1057D00022F480520284048C8288838B0D8823F407
:1057E000E6464FF6FF7303EA0525354324F40056D9
:1057F0000C8903EA043434434E8803EA0636264310
:10580000094CA04202D0094CA04205D122F48044A8
:105810008A8903EA8212224382808583C988A0F89C
:105820004010068470BD0000002C0140003401408F
:10583000828B4FF6FF7322F4006203EA01211143C9
:1058400081837047018582827047828822F07002CE
:10585000828082880A4382807047A0F84010704797
:1058600030B502881B4B1C4C98420DD0A0420BD087
:10587000B0F1804F08D0194DA84205D0184DA8426C
:1058800002D0184DA84203D122F070054A882A435D
:10589000154DA84206D0154DA84203D022F44075FC
:1058A000CA882A4302808A8882850A8802859842AB
:1058B0000AD0A04208D00E4A904205D00D4A90422C
:1058C00002D00D4A904201D1097A018601218182DC
:1058D00030BD0000002C01400034014000040040B5
:1058E00000080040000C0040001000400014004080
:1058F0000040014000440140004801404FF6FF7164
:10590000818000210180C18041800172704700299F
:10591000018802D041F0020101E021F00201018082
:1059200070470029018802D041F0040101E021F014
:105930000401018070470000234810B590F8201042
:10594000026801F01F00214951F82000204902425D
:10595000086802D040F4803001E020F48030086014
:10596000C1031C484FF0000303D51B4991F8651093
:1059700039B31A4A01881488611A89B201240F299F
:105980000BD3118801808168002900DA4942062979
:1059900003DD13490978022905D0417F012906D08A
:1059A0001188418010BD4477C377118841804188B8
:1059B0001288511A89B240F21A629142F2D3C47726
:1059C00010BD437710BD0000F4050020448F00088F
:1059D000B4020020E80C0020200D00202007002049
:1059E000170700202DE9F04FDFF8B8B16A48DFF85B
:1059F000AC91DFF8ACA190F80EC0BBF91A70BBF9FE
:105A00001C60BBF91850BBF96C10BCF1070F48D2F1
:105A1000DFE80CF08D041A30485E7600D9F80020DB
:105A20008284DAF80020C284828CC38CA7EB8202C5
:105A300012B2A6EB83034A431BB2594342F3CF226F
:105A400041F3CF23D11870E0D9F800204284DAF86E
:105A50000020C284428CA5EB820213B2C28C4B435D
:105A6000A6EB820212B243F3CF24514341F3CF237A
:105A7000E11814E0D9F80020C284DAF8002042844A
:105A8000C28C438CA6EB820212B2A5EB83031CB23C
:105A90004A43614342F3CF2341F3CF2419194942CA
:105AA0000AB244E0D9F800208284DAF80020428467
:105AB000828C438CA7EB820212B2A5EB83034A438C
:105AC0001BB2594342F3CF2241F3CF24111914E002
:105AD000D9F800204284DAF800208284428C838C3A
:105AE000A5EB820212B2A7EB83034A431BB242F337
:105AF000CF24594341F3CF22A11849420BB216E0FB
:105B0000D9F80020C284DAF800208284C28C838C09
:105B1000A6EB820212B2A7EB83031CB24A4342F304
:105B2000CF23614341F3CF22991849420CB2BBF90C
:105B30001E50594605F21E56A64201DACE8306E0F3
:105B4000A5F21E55A54201DDCD8300E0CC83B1F95D
:105B5000204004F21E55954201DA0D8406E0A4F2BD
:105B60001E54944201DD0C8400E00A84B1F9222025
:105B700002F21E549C4202DAABF8224008E0A2F284
:105B80001E529A4202DDABF8222001E0ABF822302F
:105B9000417B8173BDE8F08FB40200203C240140BA
:105BA0003C280140440500202DE9F04704466F4899
:105BB000704E002702786E48022AB0F9301004D0E7
:105BC000082A7BD0092A7AD0CBE0C27B022A02D1F4
:105BD000B0F840205AB1A4F8421071810423B6F9FC
:105BE00008101A460020FEF741FF3081B9E06249F3
:105BF000DFF88881496A0D14E5808068410215D577
:105C0000B4F9020040F2DA21884247DD40F26A41ED
:105C1000884204DD0823B4F942101A4660E0A0F27D
:105C2000DA20FAF7FAFB0022554B68E0C0F3C00116
:105C3000C0F30020DFF84C9181420CD1D8F8440029
:105C400040F2BA4188426DDD40F66A118842E1DCDB
:105C5000A0F2BA404FE04C480078C0060CD5D8F806
:105C6000440041F2243188425CDD41F2D471884223
:105C7000D0DC00F6DC401EE04448DFF8149190F8D8
:105C8000701001290BD090F86F00012807D041480F
:105C90000178C90746D04049098889B142E0B4F982
:105CA000020041F6DC6188423CDD42F23411884258
:105CB00012DC00F59270A0F500501CE04BE04EE0C5
:105CC000B0F91000B4F90210A0F59672914229DDE6
:105CD00000F5967291420BDDB4F9421020231A466A
:105CE0000020FEF7C3FEA4F84200002817DB1BE0EB
:105CF000081A00F59670FAF790FB00224B46FAF767
:105D0000F8FA0E22FAF764FBFAF7BEFB00B2C0F510
:105D1000804068438013A4F84200002D04DCA4F8FE
:105D2000427001E0A4F842501C48B0F90410D8F8C1
:105D30005000081A718B01EB600000B2F08200285D
:105D400000DCF782B4F94210B6F91600814200DA9D
:105D50000846708104E01248B0F87C00F9E77181D0
:105D6000378184F84070BDE8F087000017070020F5
:105D7000B402002064000020440500204C010020F3
:105D80000000794000C09240F8060020200D00205D
:105D900000C082407009002020000020EE05002095
:105DA000D40A002070B5134C40F224452946204601
:105DB00000F03EF800281BD0204600F0C7F8294626
:105DC000204600F01DF80C4C00212046FBF7D8FBC4
:105DD0002046FBF753FCC0F164000849C0B2042818
:105DE000087201D900F046F9BDE87040FBF78CBCA1
:105DF00070BD0000003801405800024080060020BD
:105E00000A0A01219140C943018070470029818914
:105E100002D041F4005101E021F40051818170472A
:105E2000002A828A01D00A4300E08A4382827047B6
:105E300030B501F01F0201240025C1F3421304FA1A
:105E400002F2012B0FD0022B0FD0838A4FEA1121CF
:105E50000088134204FA01F400EA040001D000B102
:105E60000125284630BD8389F0E7038AEEE710B5A7
:105E7000C1F3421301F01F040121A140012B07D0FF
:105E8000022B07D01430002A026805D00A4304E030
:105E90000C30F8E71030F6E78A43026010BD0000CE
:105EA00030B50446008A85B00D464CF6FF710840B7
:105EB000E98801432182A1894EF6F3100140A888A8
:105EC0002A8910436A890A431043A081A08A4FF6A9
:105ED000FF410840A9890143A1826846FEF716F8F0
:105EE0001948844201D1039800E00298A18909046D
:105EF00000EBC00101EB0010296801D5490000E06A
:105F00008900B0FBF1F06422B0FBF2F109010B094A
:105F10006FF018056B4300EB8300A3891D044FF05D
:105F2000320306D503EBC000B0FBF2F000F007002F
:105F300005E003EB0010B0FBF2F000F00F000843A7
:105F4000208105B030BD0000003801408088C0F3DA
:105F500008007047F8B501210920FDF7BFFF0121B6
:105F60008803FDF7BBFF10258DF803502020ADF806
:105F700000001A4E03248DF8024069463046FCF7B3
:105F80002DF916490C31086820F02000086018200F
:105F90008DF803004020ADF800008DF802406946FE
:105FA0003046FCF71BF948208DF803008020ADF83F
:105FB000000069463046FCF711F98DF803502801BE
:105FC000ADF800008DF8024069463046FCF706F94E
:105FD00001210420FCF754F9F8BD0000000C014039
:105FE00030B585B0FFF7B6FF00244FF4E1300090E4
:105FF000ADF808400C201D4DADF80440ADF80A0086
:10600000ADF80640ADF80C4069462846FFF748FF5A
:1060100025208DF8100004208DF811008DF8124015
:1060200001208DF8130004A8FDF73AFC012240F28C
:1060300024412846FFF71BFF01212846FFF7E6FE13
:10604000FBF78CFB012280212846FFF7E9FE0122A5
:1060500040212846FFF7E4FE012202210448FBF715
:1060600021FBFBF77BFB05B030BD00000038014091
:106070004400024070B51D4D00242878432834D1D7
:106080006878462831D1A878502807D0512805D003
:10609000812803D0892801D0212826D1144E70717F
:1060A000E9787172A81C891CFAF78AFFB072717ABC
:1060B000294409793182884217D106F10E0001780E
:1060C00041F0020101700B48016841F020010160BC
:1060D000317A0948002204E02B5D03552A55641CDF
:1060E000E4B28C42F8D38078707170BDB0070020A4
:1060F000800600200C0C0140520C002070B51D20C1
:10610000FDF7ADFBFDF730FA1D20FDF7BEFB15488E
:1061100090F82F10144D0623144C85F8381090F881
:106120003B1095F83B201143012A04D0022A07D0E6
:10613000042A0AD010E0827A8A420DD0007B09E05E
:10614000027D8A4208D0807D04E0827F8A4203D0AB
:1061500090F82000884200D12370002085F840008C
:1061600070BD0000640400204C01002017070020CF
:106170000B4800214180A0F1B8018A898280CB8937
:106180001A44C2800B8A1A4402814B8A1A44428103
:10619000898A1144818143F6FF71C18170470000F3
:1061A00004020020084940F61C72B1F90C0090422C
:1061B00002DA00F59F7005E041F2E302904201DD52
:1061C000A0F59F70C88170476400002038B513485F
:1061D000C16941F00401C1611E208DF80000022058
:1061E0008DF801008DF8020001248DF80340684607
:1061F000FDF756FB0A4984200880094947F690605C
:106200002C3108800020091F0880054914310C80BA
:10621000091F0880081F048038BD000000100240DC
:106220000008004030B420491E4A45788B7A114658
:1062300092F83B4091F83910AC4218D14BB1037938
:10624000994202D04379994201D140791AE080798C
:1062500009E08379994202D0C479A14202D182F83F
:106260002F3011E0407982F82F0030BC7047C5789C
:10627000AC42FAD16BB1C379994202D0037A994208
:1062800005D1007A82F82F0030BCFEF797BC407A27
:10629000E9E7437A9942E2D00479A142DFD0007A5B
:1062A000E1E70000640400204C010020FEE700004C
:1062B0002DE9F0470446007F012868D13548E18880
:1062C0000288511A89B2072916D30088E080B4F9F0
:1062D000000044F2DD414843401346F6D96148438B
:1062E0008013A060401000B2A0814FF08051B1FB3C
:1062F000F0F0FAF78DF82061B4F90C6096B1B4F9BA
:1063000002104DF6B05048430014A082B4F9047056
:106310004DF6B05207FB02F24FEA2245E58204D463
:10632000024603E00020E08330E0424212B22283C2
:10633000002D01DB2B4600E06B421BB2DFF85890CA
:10634000638398464FF4804AB24208DAFAF757F866
:106350002169F9F72AFFFAF77EF8801304E0002993
:1063600001DA484600E05046E083B04509DA2846A5
:10637000FAF745F82169F9F718FFFAF76CF8801376
:1063800004E0002F01DA484600E050462084BDE8D2
:10639000F08700002007002000C0FFFF2DE9F0413A
:1063A0004D484E4E00250078A6F15004022806D133
:1063B0004B4FF87B022802D1B7F8400030B1A586D8
:1063C0002564B56284F83850BDE8F081454881689D
:1063D000C068494300FB0010FBF7AEFE40F23331CA
:1063E0004843810BB4F8440043F6CC42504301EBE0
:1063F000903080B243F69911A4F8440088420BD340
:1064000039481146B0F90400884205DB97F8460088
:10641000022815D0032813D00123B4F934101A46EA
:106420000020FEF723FBA086B4F84000012301B250
:106430001A460020FEF71AFB20648003B06226E0B3
:10644000B4F8460041F69A13A0F51852663A9A42FB
:1064500009D2B4F94400214AFBF702FD206401206F
:1064600084F8380022E044F24711884212D994F8A7
:106470003800D8B11D480178491CC9B20170022901
:1064800014D30570206C10B1401E206408E084F81D
:1064900038500BE0A0F58040B0F5A47F03D2206C0B
:1064A0008003B06202E084F83850B562B4F840006E
:1064B0000A4980B20839323401F086FAB4F9000092
:1064C000B4F91810414389136180B4F91610484398
:1064D0008013A08078E70000170700204009002003
:1064E000B40200207C080020EE05002046010020B8
:1064F0000D480021A32280F82810C18381865030E6
:10650000C2600E22028241F26202426108220283CC
:10651000418341F2555282839203C0E9081240F24E
:106520008E32826081627047F008002010B504004E
:106530000B462D4AC3F1000028D56442002B12DA25
:10654000A04207DA214600F02DFA32F81000C0F51B
:10655000404041E00146204600F024FA32F81000A5
:1065600000F5004038E0A34208DA2146184600F062
:1065700019FA32F8100000F540402DE0204600F0F6
:1065800011FA32F81000C0F5803025E0002B12DA45
:10659000A04207DA214600F005FA32F8100000F5B3
:1065A000804019E00146204600F0FCF932F8100066
:1065B000C0F5004010E0A34208DA2146184600F07A
:1065C000F1F932F81000C0F5804005E053B12046E3
:1065D00000F0E8F932F81000B0F5004F01DDA0F549
:1065E000803010BD002010BD0C8B0008404380138C
:1065F000494300EBA13000220302002B14DDB3F568
:10660000001F01DC802001E04FF4005093FBF0F10B
:10661000014401EBD1714910814206D0521CD2B223
:106620000846062AF2D300E00021C80000B27047F5
:1066300002E008C8121F08C1002AFAD1704770474B
:10664000002001E001C1121F002AFBD170470000A9
:106650002DE9F047A74CA84821880288511A89B231
:106660000F297DD30088A4F13C052080288F08B134
:10667000401E288795F800C0A04ACCF3810001286D
:106680001DD0022820D0D18B9D4E9A48DFF87492FD
:10669000F388407E0027B1F5926F1CD8142818D3D8
:1066A0007820607643F01000F08040F26660A881A8
:1066B0002CF001002870D77389F8007018E0D08B97
:1066C00000EB4000C00302E0D08B8F494843010C2F
:1066D000DAE7401C04E0B1F5DB6F09D310B1401ECE
:1066E000607605E023F01000F0804CF00100287087
:1066F000B5F90200B5F914304143C3EBC303C1F34C
:106700008F31C3F3D10303EB510109B2A982904643
:10671000D28B4FF080535043B5F91620C0F38F3021
:10672000C2EBC202C2F3D10202EB500000B2E88217
:10673000AA6A42431213EA6293FBF2F22A63734A93
:106740001080A2680A44A260E1680144E160207CF4
:10675000401CC0B22074072802D942F3CF0000E0E9
:10676000C5E02883C9106983E760A76041F6C801C6
:106770002774884204DD298B654AB2FBF1F1E98177
:10678000C117890341EA9041800342F69B420023EE
:10679000F9F7C8FCA88457485E49A0F13C002A7864
:1067A000B0F906005FEA827C00FB01F14FEA214369
:1067B000C2F3810115D5012907D002290BD04FF270
:1067C000685141430914A18011E049F68C414843C6
:1067D0000014A08020E04CF6183141430914A18038
:1067E00026E001290ED0022918D0A0806B844A49E6
:1067F00048430014A4F81E00FBF752F947480088EC
:10680000C0B143E04AF65C3141430914A1804BF624
:106810002C21484300146884E383EDE74DF2AC512A
:1068200041430914A1804EF27C414143091469841B
:106830003B49DDE795F8200000BB88F80F7089F828
:106840000070B5F91A00A0F50C519F39B1F56E7FB3
:1068500018D8617FF42912D93249E8802E4AA1F86C
:10686000460050430014A880A1F84400FF2085F89A
:10687000200081F828002C493C20087006E0491CC3
:10688000617703E0607F08B1401E6077B5F91A10A8
:10689000B4F91E0081420EDDA07E7D2809D9F08862
:1068A00040F00800F0802148017821F002010170D9
:1068B0000EE0401C06E0A0F23D10814208DAA07E06
:1068C00010B1401EA07603E0F08820F00800F080B0
:1068D000B5F91810606908446061217E491CC9B28D
:1068E00021761F2903D94011A88367612776BDE867
:1068F000F08700001805002020070020B4020020C7
:10690000C00A00201707002030330100300A0020A1
:1069100074E8260BCC0E01004885010022070020F8
:10692000D0450100200D002014070020EE050020B6
:10693000024941F2F460886270470000DC040020E4
:1069400070B5164C06252078062825D2DFE800F021
:1069500003080E141A211248FAF770FB012016E002
:106960000F48801DFAF76AFB022010E00C480C303B
:10697000FAF764FB03200AE009481230FAF75EFBDD
:10698000042004E006481830FAF758FB0520207070
:1069900070BDFAF773FB2570257070BD18070020D5
:1069A000B08A0008090A05D0B0FBF1F0FF2800D931
:1069B000FF20704700207047D0E90021C368521AB9
:1069C0005A4301EBA231816041607047B0F9002069
:1069D000B0F90210B0F90630521A5A4301EBA23155
:1069E000818041807047000030B5494B1888494983
:1069F0000A8A801A85B24848484A0F2D047801F166
:106A000050001DD31D880D82117A090713D5022C61
:106A100001D0434912E0434DB0F90210B5F90050DE
:106A2000A94205DC02DA01F1020108E0458007E035
:106A3000A1F1020103E0022C02D13B490988418007
:106A4000B0F840101D88691A89B29C2949D3198869
:106A5000A0F84010916A0023B1F5804F31DB334933
:106A6000096DB1F5405F2CDD314940F26665B1F941
:106A70001010A94212DD43F69915A94202DB40F23B
:106A8000333108E040F23335A1F26661694343F2E5
:106A9000333591FBF5F1A0F8441001E0A0F8443043
:106AA0002449B2F806510978C1F381012DB100BF24
:106AB000B0F8441001F21E511CE092F84620022A60
:106AC00010D0A0F84430022C01D0A0F84430B0F926
:106AD0005C10B0F9443001F114029A420DDAA0F8CA
:106AE0005C2030BD012901D00229E1D1B0F8441069
:106AF00001F23331A0F84410E5E703F114029142AA
:106B000003DD1439A0F85C1030BDA0F85C3030BD56
:106B1000200700201400002017070020B4020020E6
:106B2000DA040020D8040020D40400204C01002006
:106B300044050020DC0400202DE9FC410121022055
:106B4000FDF7B4F901211920FDF7C8F901213C48EE
:106B5000FBF796FB4027ADF8007003248DF8024048
:106B60000420384D8DF8030069462846FBF736FBB4
:106B7000E001ADF800008DF802401C208DF8030004
:106B800069462846FBF72AFB4FF4E0712846FBF7DD
:106B9000ACFBA815ADF800008DF8024010208DF870
:106BA000030069462848FBF719FB4FF4A060FCF787
:106BB000A9FE1D208DF8040001268DF80560002532
:106BC0008DF806508DF8076001A8FCF769FE1F4993
:106BD0008C2008801D494FF6FA702C3108806E20F9
:106BE000091F0880194814300680184808300780AB
:106BF000164920310D80154AD020121D1080134AED
:106C000045F2F300183210800A1F45F25000108040
:106C10000E4A4FF6FF7038321080121D1080121D80
:106C2000108041F21B10088000F012F8FBF7DAFD2B
:106C3000064810300580001F0480BDE8FC8100007C
:106C4000000C1A0000100140000C0140000400403C
:106C500070B51D20FCF7F8FD2A4D40212846FBF7B2
:106C60003BFB840080212846FBF736FB44EA4004C6
:106C7000A9152846FBF730FB0443E0B2224C84F808
:106C80003C00FBF7B5FB0546052805D91F48C18820
:106C900041F04001C18001E084F838501C48007A7E
:106CA000000703D594F838001A490D5C4FF6FA70C6
:106CB0002063E062A06260622062E061A061164829
:106CC000606300206064206584F83F0084F8400021
:106CD000FBF73CFBA07AFF2811D0022084F83D008E
:106CE0000E480088A0662846FBF7DEFF207820F0DB
:106CF00001002070BDE870401D20FCF7BBBD0120E5
:106D0000ECE70000001001404C010020C00A002008
:106D1000B402002010930008DCFF050024040040AA
:106D20002DE9F0434E484F4902880B889A1A92B2D7
:106D30000F2A69D3098801804B49098B027D00EB3A
:106D400042029180017D491CC9B2017508295BD3BB
:106D5000002404752246017D00EB4103491CB3F970
:106D60000430C9B202EB630212B201750829F2D3F2
:106D70003E4904753E4B4A8044800E789D895FEA07
:106D8000C67C40F638694FF0030714D0A2F22B5CA2
:106D900042F6E858C44520D3A1F1020C26F00204C3
:106DA000ACF8002047750C7040F22B54A24211DA67
:106DB00045F004021EE046F001060E704A4507DD6C
:106DC00045F001029A8126F002020A70477519E027
:106DD000447517E045F002020CE04A450CDA87756D
:106DE000427D12B1521E42750CE046F002020A705A
:106DF00025F007029A8105E0B30703D5837D2BB107
:106E00005B1E837540888880BDE8F08342F6AA2324
:106E10009A4222DAB1F904302BB941F2CD05AA42E7
:106E200001DA4480EEE7134C920302EB843241F620
:106E30007244B2FBF4F214B24FF48055024644801F
:106E4000AC4200DA5580B2F90240E41A04F5A374AA
:106E5000B4F5237FD6D84380D4E74FF48043FAE7D4
:106E6000540B002020070020B4020020EE05002073
:106E7000C00A0020C8F1FFFF2DE9F0416D4CDFF89A
:106E8000B8E14FF0000594F83410C80706D094F923
:106E900038104B42002958DD0E4657E0674884F809
:106EA0003750A4F84250664A90F8380084F8400001
:106EB0001586CEF80450CEF80850624E40F2666354
:106EC000CEF80C50A4F87C3036F810005E4E768870
:106ED00030444FF6FF7606EA800024F8300B4FF07E
:106EE000806044F8040CA320208460845810A0849F
:106EF000E38440F699102085580060854FF4805057
:106F0000A08541F23330E08541F26660208641F68B
:106F10009910608641F6CC40A0864FF40050E08680
:106F200042F23330208742F26660608742F6991061
:106F3000A08742F6CC40E08782F89D5041F00100E6
:106F4000207184F84450BDE8F0811E4694F9370062
:106F50004242002801DD074600E01746F61B012EDD
:106F60000BD0002800DB02465FFA82F684F8380076
:106F700094F84F00012805D041E0002900DA1946B5
:106F8000CEB2F3E794F939305942002B01DB1846B1
:106F900000E0084694F93A20C7B25042002A01DBCB
:106FA000944600E08446BC4508DD002A00DA02462B
:106FB000D7B2002B00DA0B46D8B207E0002B00DA7C
:106FC0000B46DFB2002A00DB1046C0B204EB4000E3
:106FD000B0F9501004EB470030F9502F114449101C
:106FE000018084F84F5084F83E5084F83D5084F876
:106FF0003C5084F83B5084F83A5084F8395004EB04
:1070000046007546B0F9500024F8420FBEF804104F
:10701000C82309B26422FDF729FD6860E968401AB7
:10702000A9680844A860B5F900104843C013E86097
:10703000608788E7D40A0020DC0500204C0100208E
:10704000B40200202293000864000020F0B45448E9
:1070500090F83410C90776D0524990F84030002299
:1070600091F838108B426FD04F4CA0F872204F4DE2
:10707000E65C04468E4294F9374002D0EE5C8E42C4
:107080000FD1641C64B280F83740EB5C8B4202D1B4
:10709000641C80F8374090F937300F2B1BDD0F232D
:1070A00017E0434DEE5C434D8E4202D0EE5C8E42C3
:1070B00011D1641E64B280F83740EB5C8B4202D180
:1070C000641E80F8374090F937406FF00E039C4201
:1070D00001DA80F83730324B90F83F50393390F86E
:1070E0003740EC5490F83F305B1CDBB280F83F3007
:1070F000062B01D380F83F2090F9394090F93B30BE
:107100009C420ED190F93D40A3420AD190F93A40F9
:1071100090F93C309C4204D190F93E40A34200D10A
:10712000012280F84F201F4A80F8401090F9375014
:107130001378214A012D0DDD14465E07A46804D59D
:1071400044F0080403E028E015E024F0080494600B
:1071500080F83510B5F1FF3F0ADA5B07936802D576
:1071600023F0080301E043F00803936080F8351032
:10717000F0BCFBF7EBB890F84F1001290DD1B0F837
:10718000721043F60953491C89B2A0F87210994253
:1071900003D9A0F8722080F84F20F0BC704700009F
:1071A000D40A00204C010020049300080A93000830
:1071B000169300081C930008B402002030B5204943
:1071C000204AB1F86A301088C01A80B20F2836D32E
:1071D0001088A1F86A001C4D00204FF000432A5C83
:1071E000940903D00124B4EB921F24D1D20622D0FB
:1071F000164A52F820201268134C123434F810400A
:10720000224201EB000494F9722008D00A2A04DB20
:107210000A6823FA00F4224308E0521C09E012F144
:107220000A0F05DC0A6823FA00F4A2430A6002E0B0
:10723000521E84F87220401CC0B21128CFD330BD3A
:10724000F405002020070020108F0008109000088F
:107250002DE9F00779497A480A8903889A1A92B287
:10726000082A74D300880881A1F12C0042890AB150
:10727000521E4281734A92F82820802A67D302F076
:107280003F020A70C2890AB1521EC281B1F90620BA
:10729000902A0CDB8A46FF2A09D08146C089002843
:1072A00055D1694800230078092805D005E0BDE8DC
:1072B000F007624800F09EB90823644A92F8EA5049
:1072C0000DB143F004036248817AC90701D043F04D
:1072D0000203D2F808C05FEA0C5101D543F0010364
:1072E000176800215B4EFC0302D596F8654004B197
:1072F0008021C4885FEA446801D541F040015FEA1B
:10730000845801D541F020015FEAC47801D041F0F2
:107310001001007A400701D541F008014E4800787D
:10732000C00701D041F00401A00601D541F00101E0
:107330000020012D00D1082096F8705085B992F8F0
:107340004620022A04D0012A05D03AB108E072E0B2
:1073500040F0030004E040F0020001E040F00100D2
:107360007A0701D440F02000CCF3C0020025CCF312
:10737000002C624502D13A0700D4042596F86F200C
:10738000012A01D145F00105344A0027BC46127894
:107390003E46C2F38102012A04D0022A04D0032A05
:1073A00004D004E0022602E0042600E010262C4A65
:1073B00064060ED5214C1C342478240609D5147893
:1073C000640606D4274A40F6CC44926D6243140CFE
:1073D00005E0B2F8B62040F699146243940B4FF0E2
:1073E00008088AF80A804FF061088AF80B808AF84A
:1073F0000C308AF80D108AF80E008AF80F508AF8BF
:107400001070270A4B4083F06901414069408AF8B7
:10741000117079408AF81240614052468AF813C0D0
:1074200071408AF8146051754FF4C871A9F80E10B4
:10743000FF20AAF80600BDE8F0077047DC06002030
:1074400020070020F405002017070020B4020020C8
:10745000C00A0020200D002070090020DC0400205C
:107460004C010020140800205148816941F0FC01C2
:1074700081614FF4A060FCF745FAFBF741FAFCF795
:10748000A7FBF9F78DFBFCF79BF9FDF7F5F9FFF783
:1074900053FBFCF7DBF8FFF7DBFBFBF7A3F9454DEC
:1074A0004FF40050A5F81601FEF79AFD00214FF4A5
:1074B000FA5340F2EE220020401C80B29842FBD3E7
:1074C000491C89B29142F6D33B48002680F872608D
:1074D000F9F7FCF9F9F7A4FEFCF7AAFBF9F77CFD34
:1074E000FEF774FE102235493548F8F74CFE354C4E
:1074F000364FE08820F04000E0803348017821F0EA
:1075000020010170FA20F8814FF49670E887FFF7A8
:107510000FFA2F492F48FCF706FB2F48FCF728FBF2
:107520002E48416A88472E48416B8847FEF7E0FFA6
:107530002C48FAF7B1FA2C494220C8802B49C86080
:107540002B48F9F7AFFCA86820F48070A8603E7162
:10755000E088E0812089208260896082FAF7A2FDBC
:10756000FAF7FEFCFFF774F8FFF7DAFB00F0FAF920
:10757000FFF724FE01F002F8FEF7DEF9FAF760FBF0
:10758000FBF7B0FBFFF730FAFCF78CFDFAF7D2FF00
:10759000FBF704F800F07CF8FFF75AFE1148FAF701
:1075A00027F900F06BFAFDF7ABF9FAF7ABFACFE782
:1075B00000100240B402002044050020200D0020ED
:1075C00034060020C00A00204C01002014070020CF
:1075D000C008002090080020180400203800002077
:1075E000E4000020FC090020400700204C0400209B
:1075F000700A0020F0B523490278B0F90640002354
:107600001F4E31F81210FF2C18D0B0F904701E4D27
:10761000BC4231DA00EBE40704F00704BF7AA7406C
:107620008478FFB23CB190F801C0ACF1010C644524
:107630001FDA3C061DD455F822200DE056F8222012
:10764000116012498A79521CD2B28A71022A02D37D
:107650008370C3808B71F0BD11608178491CC9B201
:10766000817042789142F6D38370C188491CC180F1
:10767000F0BD56F82220EFE755F822201160F4E71C
:10768000F0900008228F000898900008B0060020B3
:10769000F0B561486149B0F86C200B889A1A92B233
:1076A0009C2A7BD30988A0F86C105D495D4F91F846
:1076B0002A1001F0070297F84610022A00D1491E4D
:1076C000594C80F83E104FF00203E2884FF0000161
:1076D000550401D5012236E0A489E50601D506222C
:1076E00031E0250701D508222DE0550603D44F4D82
:1076F0002D78AD0601D5042225E0150501D5072218
:1077000021E0150601D50A221DE0950601D50C22BF
:1077100019E0150701D50B2215E0550701D4D50551
:1077200001D510220FE0D50601D505220BE0650733
:1077300003D4A50701D4E40702D080F86E3007E037
:10774000920403D5032280F86E2001E080F86E10C9
:10775000374A384C92F820E0324A251FD2F808C048
:107760002D4AB2F87060721C92B2BEF1000F0DD0BB
:107770002CF4000CC7F808C090F86E70B7B11E2F3B
:107780001AD090F86F200AB325E007E04CF4000609
:10779000BE60A0F870200A2A01D22360F0BD142A2E
:1077A00001D22B60F0BDA0F87010F0BD2B60A0F8E6
:1077B000701080F86F10F0BD642E04D2A0F8702015
:1077C000322AEED3E9E7A0F87010EAE77F1C80F8D0
:1077D0006F70A0F8701090F86F20012A10D0002A66
:1077E000E9D0B0F87060761CB6B2A0F870601E2EBA
:1077F000D7D323603C2EDED9521E80F86F20D2E70B
:10780000B0F87020521C92B2A0F870202360C82AF1
:10781000D1D980F86F10C6E7F405002020070020BA
:10782000200D0020B4020020C00A00204C010020DE
:10783000DC040020141C0140F0B54248B0F84810A8
:10784000491C89B2A0F8481002297AD33E49002485
:10785000A0F848400A783D4B042A57D04FF48041A5
:10786000082A0BD0A0F10C02B2F900208A4200DAFB
:107870001146B3F980208A4200DA1146344A9269EF
:107880008A4200DA11B2418282881D8AC2EB8502E7
:10789000304D12B22D78C5F381062A4D44F65516A7
:1078A0007243B5F9765092126A431213C260866829
:1078B0001546C6EBC60642F3D102F60202EBA6322B
:1078C0008260C66C1644C664B0F850707F1CBFB2AC
:1078D000A0F85070B7F5806F04D3B6120682A0F8F6
:1078E0005040C464891A1C4EC26A724340F2555615
:1078F0004E4302EB4602466A32444262B3F93030EC
:10790000B2EB034F06DD1A04426206E01349B1F9F7
:107910000410B3E7002A00DA4462C162104990F80B
:107920003D2091F838108A420BD080F83D10B0F815
:107930004210A0F84410B0F84010A0F84210A0F88F
:107940004050F0BD4405002017070020B40200207D
:10795000B80C0020DC040020C3F5FFFFD40C00208D
:107960004C01002015481649B0F85A200B889A1A85
:1079700092B20F2A20D30988A0F85A10B0F900104B
:107980004AF68C4251430914A0F86C100D494FF48B
:1079900080420B78A0F10C01022B06D1B1F9003026
:1079A000934202DA1B1D0B8000E00A800021A0F840
:1079B000601020F85C1F42807047000044050020E2
:1079C00020070020170700204FF6FF7202EA80020E
:1079D00010F4404315480ED0B3F5804F14D0B3F5E2
:1079E000004F4FEA122216D0C2F5807330F81330E0
:1079F0005B424B8005E0120A30F812304B80C2F532
:107A0000807230F812000FE0120AC2F5807330F86D
:107A100013304B8005E030F81230C2F580725B42C3
:107A20004B8030F812004042088070470C8D0008EF
:107A3000104A518A908AD28A16384639A2F1110228
:107A400000D54942002A00DA52421144002800DAE7
:107A500040420844084943F6284300B2B1F93620B1
:107A60005A43921340F2D733584302EBA030C886F2
:107A700070470000B402002044050020F0B5904992
:107A800090480A8903889A1A92B23E2A1ED3008827
:107A9000088101F138004FF4FA63428A9A4202D217
:107AA000521C428200E04382874A92F82220802AB8
:107AB0000CD302F03F020A70B1F90620402A06DB1F
:107AC000FF2A04D0C2883AB1521EC280F0BDBDE880
:107AD000F0407B48FFF78EBD428A9A42F6D3077882
:107AE0004FF0010E3A074FF0FF055BD5847A40F264
:107AF000DC52630708D444F004038372C28081F827
:107B00000BE081F80AE04CE04378072B05D0032B0B
:107B100003D0052B01D0062B07D1660605D444F00F
:107B200040038372C280052239E0654A5FEA437CE4
:107B300002F138024FF42076127A0DD55FEAC26C5A
:107B40000AD45FEA446C07D442F0100202723A068B
:107B500028D4C680192222E0DF0709D0970707D46E
:107B6000670605D442F002020272C680042216E0C3
:107B70009F0709D5170707D4670605D442F0080206
:107B80000272C68003220AE01B070BD5530709D4F3
:107B9000630607D442F004020272C6800B22CA7246
:107BA0008A72CD80494AB2F92230B2F91A7003F2D2
:107BB0003D140022A74200DB0276414E444C06F100
:107BC0003806A479B6895FEAC46C06F101064FF461
:107BD000C874B6B213D58681B6F57A7F05D9017A15
:107BE00021F0800101728281F0BD037A1E06FBD470
:107BF000828143F080020272C480112035E09F42EE
:107C000016DA037E052B13D28681B6F5487F04D998
:107C10008281027A22F040020272027A5606E3D48E
:107C20005B1C037642F040020272C48002201CE01A
:107C3000284B1C89C4F3C006C4F3002740F2EE248D
:107C4000BE4216D11E78360713D4427E012ACBD10C
:107C5000428BB2F5167F02D2521C4283F0BD827A6B
:107C600042F002028272C4800F20C8728872CD80F6
:107C7000F0BD93F80D714FF40046012F18D1164F47
:107C800041F6583C7F6C674512DD83F80CE1134BDD
:107C90001E60C38AA34202D25B1CC382F0BD4FF4B4
:107CA000FA73C3801C23CB728B72CD80C282F0BD6D
:107CB000C2820A4883F80C21001F0660F0BD000054
:107CC000C006002020070020F4050020DC0400206E
:107CD000C00A0020B40200204C010020140801401A
:107CE0002DE9F05FFD48FE49DFF8F8A3007E0A1D8C
:107CF000131D012850465ED030F85A4F0C80418841
:107D00001180BAF85E001880FDF76CFEF64DF74C56
:107D100049F2CD32B5F91E10A183B5F9200043F622
:107D2000CC4C01EB400050430014E083B4F9223006
:107D3000B4F9206000FB03F201FB062242F38F320C
:107D40006282B4F91870704307FB0CF740F2333CC1
:107D5000BF1302FB0CF207EBA23201FB13002283DC
:107D600040F38F30A082B4F91A1043F6AE7251433B
:107D700000EB0012891302EB8010DD4F01EBA03005
:107D8000DC4E6083786C3060316930468847DA4970
:107D9000308948800846FDF707FFDFF860B3012609
:107DA0004FF000099BF8000008280CD0618F218259
:107DB00004284AD01AE030F8604F0C8041881180C6
:107DC000BAF864009FE7CE4890F93710491C0229A1
:107DD00039D890F8741019B1B4F85A00208205E02F
:107DE000618F2182A4F85A1080F87460B4F91410DD
:107DF000B4F90A00C34AF9F74DFBE062BAF916116B
:107E0000884204DDBF48E162027C91408162B7484C
:107E1000DFF8F4E2503847F2A30802784EF2461138
:107E2000002A7AD0012A79D080F800909BF80000CF
:107E300004280DD0B34AB4F91210B4F90800303A4E
:107E4000F9F728FB08E0608FC8E7686A0014E06271
:107E5000B87A002863D0AD48A3462546A062A94C55
:107E6000443C2060E86A606020461035FCF7F6F874
:107E70009E4928883C39FFF7A7FDDFF87082A8F1FA
:107E80005008D8F81410C8F87010B5F91010A06890
:107E9000B5F9123000FB01F7E268584302FB137496
:107EA00044F38F3702FB0100AF8740F38F34EC8738
:107EB000974D28466F80AC80FEF7FAF9287F08F1CD
:107EC0001805012871D0604241104DF6B350474368
:107ED00069803A142A804046A8F804408B18C38071
:107EE000891AA8F808108AF80C90B8F9043054469A
:107EF000002B00DD2673B8F90600002802DD217B87
:107F0000891C2173B8F90820002A02DD217B091D94
:107F10002173217B072979D202E007E02CE05AE0A7
:107F2000DFE801F07470886E84728600B5F91E2057
:107F300042448A420AD8B5F9202042448A4205D8F0
:107F4000B5F9222042448A427FF670AFA0F8029031
:107F5000B7F8B6204946B2F5C87F01D8467006E0AA
:107F6000B2F5487F01D8022200E0032242708AF86D
:107F70000F108BF8001025E080F80090B5F91EC0B6
:107F80004A46C4448C4509D8B5F920C0C4448C4540
:107F900004D8B5F9225045448D42D5D9B7F8B6106A
:107FA000B1F5C87F02D8467007E017E0B1F5487F09
:107FB00001D8022100E00321417042808AF80F209D
:107FC0008BF80020BEF8061041F40061AEF80610F0
:107FD000F9F7B8FF2AE74FF4AF703DE74C484DF68C
:107FE000B352B0F92030594249106980B0F91E00EF
:107FF000504302142A804046A8F804306EE705E09A
:10800000667303E0022100E0032161739BF8001016
:10801000404E0129404F617BDA460DD007297DD2C1
:10802000DFE801F07CFDFCFBFAF9F8000421ECE745
:108030000521EAE70621E8E70729F0D2DFE801F0A9
:108040006E0429799ECCF80001461846FBF752FDD4
:108050002860B5F9020040F68151484380136880DA
:10806000B5F9001040F68152514389132980421816
:10807000A2F68152B8F80E305242C3EB620212B23D
:10808000A8F80C20002A01DCA8F80C90B8F80C2005
:1080900067E1404201B2504200B2FBF72BFD28607D
:1080A000B5F9020040F68151484380136880B5F964
:1080B000001040F681525143891329804218A2F6DC
:1080C0008152B8F80E305242C3EB620212B2A8F8E5
:1080D0000C20002A01DCA8F80C9020E0FC0900200C
:1080E000342C0140B402002044050020640000202C
:1080F0004C0100204C040020080400201707002039
:10810000D40A0020C0080020C00A0020A2FEFFFF01
:10811000300A00200024014000280140C6E0B8F8E1
:108120000C204CE13046F8F799FD01231A4607214F
:10813000B1E019461046FBF7DDFC2860B5F90200F6
:1081400040F68151484380136880B5F9001040F62D
:1081500081525143891329804218A2F68152B8F8FE
:108160000E305242C3EB620212B2A8F80C20002A71
:1081700001DCA8F80C90B8F80C204DE159424042BF
:1081800009B200B2FBF7B6FC2860B5F9020040F670
:108190008151484380136880B5F9001040F6815240
:1081A0005143891329804218A2F68152B8F80E3043
:1081B0005242C3EB620212B2A8F80C20002A01DC82
:1081C000A8F80C90B8F80C2056E13046F8F746FDB8
:1081D00001231A4605215EE01146FBF78BFC28605F
:1081E000B5F9020040F68151484380136880B5F923
:1081F000001040F681525143891329804218A2F69B
:108200008152B8F80E305242C3EB620212B2A8F8A3
:108210000C2006E06FE143E114E1E5E0B5E088E021
:1082200006E0002A01DCA8F80C90B8F80C204EE11A
:10823000504201B2584200B2FBF75CFC2860B5F92D
:10824000020040F68151484381136980B5F900006E
:1082500040F681525043801328800A18A2F68152BA
:10826000B8F80E305242C3EB620212B2A8F80C20EA
:10827000002A01DCA8F80C90B8F80C20A4F85C20C7
:108280001144A4F85E10084455E13046F8F7E6FCC6
:1082900001231A4606213846F8F7E0FC0121304652
:1082A000F8F752FC01213846F8F74EFCB04EBAF808
:1082B000080055463080BAF80A007080BAF81000FD
:1082C000B0803046F9F7F6FAB4F85A00F18808445D
:1082D000A4F86000B4F85C0031890844A4F8620096
:1082E000B4F85E0071890844A4F86400317EA148A6
:1082F000012978D034F85A1F018061884180A18813
:1083000081809C49028808310A8042884A8080889E
:1083100088809848896A0830884795F83E00002888
:108320007ED0F8F7ABFE15F83E0F401E2870BDE872
:10833000F09F01461846FBF7DDFB2860B5F9020007
:1083400040F68151484380136880B5F9001040F62B
:108350008152514389134218A2F681525242298018
:108360005208A4F85E201044A4F85C000844A4F865
:108370005A0000213046F8F7E7FB00213846F8F7AD
:10838000E3FB01231A460621CCE6404201B25042EB
:1083900000B2FBF7AFFB2860B5F9020040F681514F
:1083A000484380136880B5F9001040F6815251436C
:1083B00089134218A2F68152524229805208A4F829
:1083C0005E201044A4F85A000844A4F85C00002180
:1083D0003046F8F7B9FB00213846F8F7B5FB012322
:1083E0001A4605219EE6B4E019461046FBF782FBCB
:1083F0002860B5F9020040F6815148438013688037
:10840000B5F9001040F68152514389134218A2F683
:108410008152524229805208A4F85A20104400E0A8
:108420009AE0A4F85E000844A4F85C0000213046FD
:10843000F8F78AFB00213846F8F786FB01231A4635
:108440000721C2E65942404209B200B2FBF752FB93
:108450002860B5F9020040F68151484380136880D6
:10846000B5F9001040F68152514389134218A2F623
:108470008152524229805208A4F85A201044A4F88C
:108480005C000844A4F85E0000213046F8F75CFB6D
:1084900000213846F8F758FB01231A46062194E6D6
:1084A0001146FBF727FB2860B5F9020040F6815121
:1084B000484380136880B5F9001040F6815251435B
:1084C00089134218A2F68152524229805208A4F818
:1084D0005C201044A4F85A000844A4F85E0000216F
:1084E0003046F8F731FB00213846F8F72DFB012321
:1084F0001A460521C9E6504201B2584200B2FBF7C4
:10850000F9FA2860B5F9020040F68151484380131A
:108510006880B5F9001040F6815251438913421822
:10852000A2F68152524252082980A4F85C201044DD
:10853000A4F85E000844A4F85A0000213046F8F779
:1085400003FB00213846F8F7FFFA01231A460721FA
:108550009BE634F8601FCFE607480088A0F5D041BD
:1085600068393FF4E4AEBDE8F05FF9F73DBC0000C8
:10857000FC09002030000020182C01402DE9F041BA
:10858000964C9748B4F862100288511A89B20F29A4
:108590006FD30088A4F8620092480088DFF8488210
:1085A000C0074FF000054FF0010741D08D4AD4E9D4
:1085B0000C1024321388B1EB530F02D21288511AD7
:1085C00008444FF4F371884200D208468749B1FB52
:1085D000F0F0616CC1F35101084406466064F7F79E
:1085E0001CFF0022824BF7F784FE4FF04042814B84
:1085F000F7F77FFE0E22F7F7EBFEF7F745FFA4F83B
:10860000AC0094F86D00401CC0B284F86D000828DE
:1086100034D3724898F84620001F03789A4201D05C
:1086200002704580744A1378744A23B1458021E072
:108630006564256568E0D8F89410A1F5FA618E426A
:1086400011DDE16D8B1C9E4205DDB0F902100A2997
:108650000DDA491C06E08E4205DAB0F90210002955
:1086600008DD491E4180B0F902000A2802DB1770BC
:1086700001E0AFE01570E66584F86D5060484FF496
:10868000A5420178C1F38103012B59D044F2506116
:108690002181A4F8A820B0F9243089B24B439B1360
:1086A000A4F8A430B0F90E00D4F850C07043B0FB69
:1086B000F1F35449CCEBCC0C4FEACC2C0988C3F332
:1086C000D10303EB9C33B0032365B0FBF1F14E4BB8
:1086D000C908B3F846C0CCEBCC0C4FEACC2C01EB6C
:1086E0009C31A3F84610F117890341EA9641002313
:1086F000F7F718FDB4F8AA10C1EBC101C902C00810
:1087000000EB9130A4F8AA00616C206F0844206748
:1087100094F87420521CD2B284F87420082A05D32D
:10872000C008A4F8760084F8745025673748384E9E
:10873000C3885A0630D498F80F20022A03D029E0C3
:1087400045F6C051A4E7B26840F69916B24221DD61
:1087500094F8382094F88E60B2420CD084F88E20C1
:1087600094F83D2002F00106C2F34002964202D185
:10877000A4F88A5004E0B4F88A20B2F5966F05D2C6
:10878000B4F88A00401CA4F88A0005E043F0800297
:10879000C28001E0A4F88A50104894F83F30B83005
:1087A0000C2B01D2C57400E0C774194A41F2482667
:1087B00041F2504C92F83C400B4A0C2BB2F882200C
:1087C0000AD3B14208DB012C06D0614502DD002A44
:1087D00000D18774BDE8F0818574FBE74C0100206F
:1087E0002007002000040040B40200204564BD01C1
:1087F00000209C40133B3340060400200704002067
:10880000DC04002044010020F0080020C00A002001
:10881000440500202DE9F041384C394E394F20787D
:1088200041F23331C2074FF000050CD0A28962B388
:1088300094F90700002800DA4042C0B2032829D288
:1088400040F2AE702AE0A570E5732F4AE571A5816C
:1088500092F83830237220F00800A18040F0020026
:1088600020703D867560B560F560116D490005D0DA
:1088700041F68461A18140F010002070C0B240F048
:10888000010020706574BDE8F081658120F0100062
:10889000207015E0042803D240F6510060810FE0FB
:1088A000052802D240F69910F8E740F6CC42062897
:1088B00003D3072801D3082801D2628100E0618137
:1088C00097F89D0098B9B088102301B2B4F90A0056
:1088D0003622FCF7CBF87060F168401AB1680844A2
:1088E000B060B6F900104843C013F0603886388E87
:1088F00010B10120A070C6E7A570C4E7D40C002019
:10890000A0060020B40200204C0100202DE9F04117
:10891000554C2678F0077CD05448217A544D90F875
:10892000380081427BD0534A2346DFF84CC1575C64
:1089300093F90E2093F90730874203D01CF8017099
:10894000874213D146F002065B1C26705BB2E371CE
:108950001CF80110814201D15B1CE37194F90710EE
:10896000062901DD0621E171521C1CE0434F17F876
:1089700001C0434F844503D017F801C0844513D18B
:1089800026F002065B1E26705BB2E371795C8142C1
:1089900001D15B1EE37194F907306FF005018B4242
:1089A00000DAE171521EA273207294F907108A1C3A
:1089B000042A02D941F68462A2812C4A0129127844
:1089C0000ADD2B4B56079B6802D543F0080301E0F4
:1089D00023F00803AB606070B1F1FF3F09DA510783
:1089E000A96802D521F0080101E041F00801A96061
:1089F0006070F9F7ABFCA078012810D1214880689D
:108A0000A3280CDA94F90700022803DD0220E071A4
:108A100005E01EE06FF00101884200DAE171A089F3
:108A2000002630B1401E0004000CA08101D1E67187
:108A3000A673E87B04280CD0B5F9301051234122ED
:108A40000020FCF713F82886002802D1E07B10B143
:108A5000A670BDE8F0810C4806700C4806702078BE
:108A600020F001002070F4E7D40C00204C0100201D
:108A7000B4020020049300080A930008169300082B
:108A80001C9300084405002034070020170700202D
:108A9000173E573CBB3A3E39DD3794366135413499
:108AA00033333532443161308A2FBD2EFB2D412DB9
:108AB000441458585870111158585870411158584A
:108AC00048701114485858701411584858700000D4
:108AD0000102030405000500010203040104000370
:108AE00005020000F001000036010000F80000005F
:108AF000BA0000007C0000007C0000007C00000048
:108B000041141411111444111414411100002900CE
:108B100052007B00A400CC00F5001E01470170014B
:108B20009901C201EA0113023C0265028E02B602FB
:108B3000DF020803300359038203AA03D303FB03B4
:108B400024044C0475049D04C504EE0416053E057A
:108B500067058F05B705DF0507062F0657067F0651
:108B6000A706CE06F6061E0746076D079507BC0743
:108B7000E4070B08320859088108A808CF08F6084E
:108B80001D0944096A099109B809DE09050A2B0A79
:108B9000520A780A9E0AC40AEA0A100B360B5C0BCA
:108BA000820BA80BCD0BF30B180C3E0C630C880C3E
:108BB000AD0CD20CF70C1C0D410D650D8A0DAF0DDF
:108BC000D30DF70D1C0E400E640E880EAC0ECF0EAA
:108BD000F30E170F3A0F5E0F810FA40FC70FEA0FA6
:108BE0000D103010531075109810BA10DD10FF10D2
:108BF0002111431165118711A911CA11EC110D1230
:108C00002E12501271129212B312D412F4121513C2
:108C10003613561376139613B713D713F613161489
:108C20003614561475149414B414D314F214111584
:108C300030154E156D158C15AA15C815E7150516B6
:108C4000231641165F167C169A16B716D516F2161D
:108C50000F172C17491766178317A017BC17D917BA
:108C6000F51711182E184A18661881189D18B9188A
:108C7000D418F0180B19261942195D197819921990
:108C8000AD19C819E219FD19171A311A4C1A661ACA
:108C9000801A991AB31ACD1AE61A001B191B331B36
:108CA0004C1B651B7E1B971BAF1BC81BE11BF91BD5
:108CB000121C2A1C421C5A1C721C8A1CA21CBA1CA4
:108CC000D21CE91C011D181D301D471D5E1D751DA0
:108CD0008C1DA31DBA1DD01DE71DFD1D141E2A1ECF
:108CE000401E571E6D1E831E981EAE1EC41EDA1E29
:108CF000EF1E051F1A1F2F1F451F5A1F6F1F841FAE
:108D0000991FAE1FC21FD71FEC1F00200000640078
:108D1000C9002D019201F7015B02C00224038903FF
:108D2000ED035204B6041A057F05E3054706AB06BA
:108D30000F077307D7073B089F0802096609C9098F
:108D40002D0A900AF30A560BB90B1C0C7F0CE20C8F
:108D5000440DA60D090E6B0ECD0E2F0F900FF20FC6
:108D60005310B41015117611D71138129812F81249
:108D70005813B81318147714D61435159415F31521
:108D80005116B0160E176B17C91726188318E0185E
:108D90003D199919F519511AAD1A081B631BBE1B11
:108DA000181C731CCD1C261D801DD91D321E8A1E49
:108DB000E31E3B1F921FEA1F41209820EE20442112
:108DC0009A21EF2145229922EE2242239623E9237C
:108DD0003C248F24E22434258525D725282678268F
:108DE000C82618276827B72706285428A228EF285E
:108DF0003D298929D629222A6D2AB82A032B4D2BF1
:108E0000972BE12B2A2C722CBB2C022D4A2D912D55
:108E1000D72D1D2E632EA82EEC2E302F742FB82F99
:108E2000FA2F3D307F30C030013141318131C131C5
:108E300000323F327D32BA32F73234337033AC33E2
:108E4000E73322345C349534CE3407353F357735FB
:108E5000AE35E4351A3650368536B936ED3620371C
:108E600053378637B737E937193849387938A8384A
:108E7000D738053932395F398B39B739E2390D3A8C
:108E8000373A603A893AB23ADA3A013B283B4E3BEC
:108E9000733B983BBD3BE03B043C263C483C6A3C72
:108EA0008B3CAB3CCB3CEA3C093D273D443D613D1E
:108EB0007D3D993DB43DCE3DE83D013E1A3E323EFA
:108EC000493E603E763E8C3EA13EB53EC93EDC3E0C
:108ED000EF3E013F123F233F333F433F513F603F4F
:108EE0006E3F7B3F873F933F9E3FA93FB33FBC3FD1
:108EF000C53FCD3FD53FDC3FE23FE83FED3FF13F8F
:108F0000F53FF93FFB3FFD3FFF3FFF3FFF3F0000C5
:108F1000E7382C35002020EF20372023332026206F
:108F2000210000800200040008001000000200047C
:108F300000080400000200040008001000200040A7
:108F400000800400000000800000004000000020BD
:108F500000000010000000080000000400000002F3
:108F60000000000100008000000040000000200020
:108F700000001000000008000000040000000200D3
:108F8000000001000080000000080140000C0140CA
:108F9000000C0140000C0140000C0140000C01409D
:108FA000000C0140000C0140001001400010014085
:108FB000001001400010014000100140001001406D
:108FC000001001400010014000140140040801405D
:108FD000040C0140040C0140040C0140040C01404D
:108FE000040C0140040C0140040C01400410014039
:108FF000041001400410014004100140041001401D
:109000000410014004100140041001400414014008
:1090100008080140080C0140080C0140080C014000
:10902000080C0140080C0140080C0140080C0140EC
:1090300008100140081001400810014008100140CC
:1090400008100140081001400810014008100140BC
:10905000081401400C0801400C0C01400C0C0140AC
:109060000C0C01400C0C01400C0C01400C0C01409C
:109070000C0C01400C1001400C1001400C10014080
:109080000C1001400C1001400C1001400C1001406C
:109090000C1001400C14014010080140100C01405C
:1090A000100C0140100C0140100C0140100C01404C
:1090B000100C0140100C0140101001401010014034
:1090C000101001401010014010100140101001401C
:1090D0001010014010100140101401400000000069
:1090E0000000000000000000000000000000000080
:1090F00014080140140C0140140C0140140C0140F0
:10910000140C0140140C0140140C0140140C0140DB
:1091100014100140141001401410014014100140BB
:1091200014100140141001401410014014100140AB
:1091300014140140000000000000000000000000C6
:109140000000000000000000FFFFFF0F0FFFFFFF07
:10915000FFF0FFFFFF0FFFFFFFFFF0FF0FFFFFFF1D
:10916000FFF0FFFFFF0FFFFFFFF0FFFF0FFFFFFF0D
:10917000FFF0FFFFFF0FFFFFFFFFF0FFFFFF0FFFFD
:10918000FFFFFFF0FFFFFF0FFFF0FFFF00000040B9
:109190004000000000040000004000000000040047
:1091A0004000000000040000004000000004000037
:1091B0004000000000040000004000000000040027
:1091C0000000400000000004000000400004000017
:1091D0000000008080000000000800000080000007
:1091E000000008008000000000080000008000006F
:1091F000000800008000000000080000008000005F
:10920000000008000000800000000008000000804E
:109210000008000000000020200000000002000004
:1092200000200000000002002000000000020000FA
:1092300000200000000200002000000000020000EA
:1092400000200000000002000000200000000002DA
:10925000000000200002000000000060600000002C
:109260000006000000600000000006006000000032
:109270000006000000600000000600006000000022
:109280000006000000600000000006000000600012
:1092900000000006000000600006000000800200E0
:1092A000040008001000000200040008040000028E
:1092B00000040008001000200040008004000000AE
:1092C000FF7FFFFFFDFFFFFFFBFFFFFFF7FFFFFF3C
:1092D000EFFFFFFFFFFDFFFFFFFBFFFFFFF7FFFFBC
:1092E000FBFFFFFFFFFDFFFFFFFBFFFFFFF7FFFFA0
:1092F000FFEFFFFFFFDFFFFFFFBFFFFFFF7FFFFF6E
:10930000FBFFFFFF01020304050002030405000147
:109310000304050001020500010203040405000125
:10932000020355050010AA1A55250030AA3A00007C
:10933000AA0A55150020AA2A5535FF3F5C9300085C
:10934000000000204C070000E406000848940008D4
:109350004C0700204C0A0000406600084502040645
:10936000082D010203040405480607080913912B80
:109370001B08A504211355152A4006190801A71337
:10938000B73D1B08DD041AD704012073286E1702AD
:109390000604050103148020FF8BAA0A0201A4150C
:1093A000AA0A551500085920AA2A5535FF3F072D4E
:1093B00003010504060203127C1573FFFF04FF80FE
:1093C00080010129025F6402130A13B9695208126D
:1093D00001100C0504060203010103070505280B13
:1093E000010203040206070303040C3D07060405FB
:1093F00009191F191904310506060B14AA1A02319E
:109400002E40FD3969260211042F405F020C2640D0
:109410005B262ACD55155515123902017F0316D04A
:10942000071AFF01013B0261AA6C080108A809168E
:10943000C491220312100A17401C12600A16901BD6
:08944000014D13CD6902000883
:020000040800F2
:10FC00004A46545A594D46312D4E3330202020203B
:10FC1000050406020301AA0AAA0AAA0AAA0AAA0A4B
:10FC2000AA0ADE3F00100000FF0131000201664613
:10FC300000400040513800400040004000400101B9
:10FC400000400040FF387B257B257B25FF003333B8
:10FC50000201401F00016626B81E6626FFFFFFFF57
:10FC6000FFFF01010100010000000200000202008C
:04FC70000000AA5591
:04000005080000ED02
:00000001FF
